:020000040000FA
:80000000FFFF62FF3900FFFFFFFFFFFFFFFFFFFFFFFFFFFFFFFFFFFFFFFFFFFFFFFFFFFFFFFFFFFFFFFFFFFFFFFFFFFFFFFFFFFFFFFFFFFFFFFFFFFFFFFFFFFFFFFFFFFFFFFFFFFFFFFFFFFFFFFFFFFFFF800C9001324006C840110051200A4481A80255048A4011300245804C9001000000000000000000000000000000000C90013200C0
:8000800026C80419280245C00814A8225004401488320245A0089001C0FB0017E0025C800B70012A800A50012A4005B4800A50012A4005A8003FE0020000000000000000000000000000000012E0025C001DF0032E4005A80015A00554800AA002544005A80015E00298FF0000000000000000000000000000000000000000000000000033
:80010000000000000000000000000000000000000000000000000000000000000000000000000000000000000000000000000000000098FF0000000000000000000000000000000000000000000000000000000000000000000000000000000000000000000000000000000000000000000000000000000000000000000000000000009850
:80018000FF00012000048000100000000000000000000000000000000000008021200000000000000000000000000000000000002000050010108202000000000000000000000000000000000000200030FC1601800401001010000000000000000000000000000000000000008480040000000000000000004000000000000000C00010A1
:800200000020601000000000000000000000000000000000000000A080C5FD0000000000000002000008000000000400000000000000000000200000000000000000000000000000000000002000000000D0001A40000000010000008000000002400308040120000000D8FC000000000000001800000000000000000000000000000000B5
:800280000000000000000000000000000000000000000000008001000000C00018000000000C0000000000000000000300100000000000C8FD000000000000001E000058000000000000000000000000000000E0410000000000000000000000000000000000E001000000E0001CC00000000C0000008001000004000018000240000000A2
:80030000E8FF000000000000000000002000000000B008000000000000000000001000000000000000000000000000000000000000000000D0001A00000000001000000000000002000060100120000000A0FF000000000000000C00003000000000801000000000000000000080450000000000000000000000000000000000C000000031
:800380000000080109A30000000000000026020098000851000C8105000070FB0000000000000010000040000000003C00000000000000000000E00100000000000000000000000000000000000001000000200004800300000D040000000700001C440040000EC0810000E8FE0000000000000010000040000000003000000000000000B0
:80040000000000804100000000000000000000000000000000004001000000000000000300000C0000000006000018000340000C80010000E8FE000000000000000800002000000000300900000000000000000080090000000000000000000000000000000000800000000000000200030000000000000006000018000320000DA0010039
:800480000058FA0000000000000002000008000000000400001000004000000001200000000000000000000000000000000000002000000000D00052400000004100000000001000024003081401200000004CFD000000000000000000000000000000000000000000000000000000000000000000000000000C000000000000000600007B
:800500000000C0000808000000080400000000000000000000000000000000F8FD0000000000000016000058000000000000000020000000000000000001000000000000000008000000000000006401000000E0001880000000040000000000002004000018100240000000F0FD000000000000000800002000000000B00800C002000015
:800580000000000C810900000000000000000000000000000000008000000000D00088440000008C0800000000C0000200136A0001200000002BFB000000000000000C00003000000000001200001000000302000001840000000000000000000000000000000000C00000000000049800630000080000000000004218000350000C803116
:80060000000069FE0000000000000010000040000000003C0000F00000C00300000FE0010000000000000000000000000000000000000100000020801E84030000090000000000F0001C440040000EC201000068F9000000000000001000004000000000300000C00000000300000C800100000000000000000000000000000000004001C2
:8006800000000000001804030000040000000000C00018000040000C80010000A3F8000000000000000800002000000000300800C02000000300000C82410000000000000000000000000000000000800000000000009C40030000040000000000C0201A000320000CA001000028FA1000040000104402000008000D0000040000100000A3
:8007000000000000002000000000000000000000000000000000000020000000009020424400000001010000000010000240030800012000000020F80000000000000000000000000C000000000000000000000000000000000000000000000000000000000000000000000000004000000000000008000000000000000000000000000017
:80078000000000D8FF0000002000000016000058000F000000000000200000000000000000010000000000000000000000000000000060010000008080088400000004000000000000000600007000024000000020FD0C00300100404208000020000D0000000000C0020000000000008009000000000000000000000000000000000080DF
:8008000000000000C00400400000002C040000000000000000036C000120000000E0F9040000100080040C00003000400200000200000800000000000000900000000000000000000000000000000000C00000000080085800030100080000000000000818010350008C8001000040FC00003C0000704010000040000300000C1000F04037
:80088000000000000000E00100000000000000000000000000000000000001000000F0201E8803000009000000000030401C440020000EC2410000D8F80C00300000C0001000004000000000300000C000000000000000800100000000000000000000000000000000004001000000C0001804030000040000000000C02018000020000C7E
:800900008001000070FF0000B0080040400800002000010000300500C022000000000000804500000000000000000000000000000000008000000000E0249840030000040000000000C0041A000340000C8001000050FC0000041200101802000008000D00000400005008000000000000200000000000000000000000000000000000001C
:8009800020000400009080024400000021040000000000000240032800012000000004F90000000000000000000000000C000030000040200000000000000000000000000000000000000000000000000000000000000000000000000008000000000000001800004000000000000008FC0000001000000016000058000F00000000000040
:800A000000000000000000600000000000000000000000000000000000006001002000C000008400000004040000000000001E00003000034000000098FC0000900000400209000020000D00000041000080000000000000000000000000000000000000000000000000008000300200800401410000000C0000000000000002000B410089
:800A8000002000000033F90000A0080080420C00003000400000300800000400000000000000400000000000000000000000000000000000C000800000C020000523000008000000000000000C000330002C80110000A9FD00001C000070001000004000030200340000304000000000000060000000000000000000000000000000000071
:800B00000000013C2000F0000680830000090000000000000010400050000EC241000040FD0000300000C04010000040000000003000008000000000000000804100000000000000000000000000000000004001300000C0200004030000040000000000000010000020000C8001000093F800009008004000080000200000000000000093
:800B80008022000000000000800100000000000000000000000000000000008000300A00C0084800030000040000000000000008000340000C8001000088FD3000940000500802000008000D00000406001004000000000001208800000000000000000000000000000000002000000000D0001A40000000010400000000108842440368D2
:800C000000012000000034FC0000100800404000000000000000002000000040000000000000000000000000000000000000000000000000000000000000C0001800000000080000000000000000000060000000000000A8FD0000001000000016000058000000001020000000000000000000000000000000000000000000000000000098
:800C800000006001000000E0001C80000000040000000000000006040070000240000000E8FC0C0080000000420800002000400400B00000408000000000000C812000000000000000000000000000000000008000000000D0001A400000002C08000000000044580023690001200000002BFF840501120000440C000030008C0000000023
:800D000000800200000000008000050000000000000000000000000000000000C000000000000880000B0000080000000000808414000300014C8805000079FCE0010C0000300010000040000D0400040000702000000000000FE4400000000000000000000000000000000000000100000020400488830000090000000000300010400069
:800D800010100EC041000070F88C01200800800010000040000C0000000000C00000000000000C82010000000000000000000000000000000000400100000000000000030000040000000000000010000000000C800100002BFD8001A00000804808000020000C0000000000402000000000008C80400000000000000000000000000000A6
:800E0000000000800000000000000200030000040000000000004208000300000D80010000B8F80000040000504802000008004504000402001000004000000001201001000000000000000000000000000000002000000000100002400000004104000000001000024503080001200000009CFE00000000004000000000000008000020AB
:800E8000080000000000030000000000000000000000000000000000000000000000000000000000000000000008000000000000000000000000000000000030F80000002000000016000058000C000010000000000000000100000000000000000000000000000000000000000060010000000040048000000004080000000000200604B1
:800F0000001A000240000000F8F9080030010000020900002000080800302100000000000300000C818800000000000000000000000000000000008000000000C00202400000004C0000000000C0001A000B00000120000000FBFE000000040000180C000030000000000000000004000013010020080901000000000000000000000000D6
:800F800000000000C00000000000449820130000000000000000004814000360104C8209000041FC00003C000030001000004000010000040000308000C00300000FE00000000000000000000000000000000000000001000000F0001C80830000010000000000F00010400070000EC041000078F90400300800804010000040000000008F
:80100000000000C08000000300000C820100000000000000000000000000000000004001000000C0201800030000000000000000C02010000060000C8001000033FF0000B0000080020800002000000000000000C00000800801002C808400000000000000000000000000000000008000000000C0021A00030000000000000000C0020857
:80108000000368000C8001000078FA3000040000100002000008008510000400001000024000000001A0100000000000000000000000000000000000200000800010001A400068008128000480001000024403680001200000005CFE00000000000000000000000008000020080000000000000000008040000000000000000000000000D1
:80110000000000000000000000000000180000600008000000000000000000006000000000000000FE0000002000300016000058000C0400000000300006000000000000000000000000000000000000000000000000600100000004201C800078000468000C800100000604006000036000000058FC0C003001000000080000200048002D
:8011800000202200000000000B01000C012000000000000000000000000000000000008000000046C0021A400060002C000000000000009A004360000000000000A3FE840581000000220C00003000000000000000000418022301004004880000000000000000000000000000000000C00000002002021800930044088021B01046020826
:8012000014000300010C82450000F1F9E0013C2000300010000040000100000C000030201CC00300000F600000000000000000000000000000000000000001008007F0201C8003100009C001380007304010400018100EC0010000A8FB8C01300800C0201000004000000000000000C04018000302000C0201000000000000000000000066
:801280000000000000004001000006C1001800030000048001300006C02010000000000C8001000083FB8001300000C0080800002000000000000000C00018001300000C004500000000000000000000000000000000008000000006C0481800030000048001300006C00808000300000C80010000C0FB0000040000100002000048004D0E
:8013000000000400001000004000000001A00404000000000000000000000000000000002001000000100002400008008D2000040000108802420308000120003400A0FA00000000000000000000200000040000000000000000000000008080000000000000000000000000000000000080000000000000000000000004080000000000BE
:801380000000000001000000003000D8FE0000002000F00016000058000E0200000000F00000000000000000000C000000000000000000000000000000006001000000004000C00018000C60000C0000000006C08310000260003C00A8F9000030010000220800002000410000B00800002800000000000C01880000000000000000001092
:80140000000000000000008800000000C002982000000004010000000000429A4210080001000030009AFF0000001100C0040C00003000040000800000C02400000302000004103110020000000000000001000000000000C000000000004840088B6040048001300600800014000160122C8249000688FD00003C0000F020100000500024
:801480000B00003C2000F00000C00300000F600038000400000000000010020000000000004801000000F0001E8003700007C081380000304010800270000EC0010C00C0FF0000300800C0201000002000040000300800C04000000300000C02013180040000000000005002000000000000C800000000C0201804036000048001300000C6
:80150000008010000160000C80010000C9F80000300100C0020800004000090000300100C00200000300004C001130000400000000000000020000000000000001000000C0049800036000048001300000000808000268000C8001000060F81000000000000000000000000000000000000000000000000000000000000400000000000077
:801580000002000000000000000000000000000800000000000000000000000008000020000000000000A4FD20000480001000024000080001200004800010000240000800012000040000000000000000000000000000000020000480001000000000080001200004800010000040000000000000040038FA00000000000000000000000F
:801600000000000000000000000000000000000000000000000000000000000000000000000000000000000000000000000000000000000000000000000000000000000098FF2C0004800010000240000800813000048000100002400008000120000400000000000000000000000000000000200004800010000240000900012000048071
:8016800000100002400008000124800400B3F8040000000000000000000000000000000000000008080000000000001040000000000000000000000000000000808000000040400008012420008080101002020000080101200484800000D9F820000480001000005000004000200004800010000040000800012000000000000000000083
:8017000000000000000000000000000480000000000000000001000000000010000000000000000000040000FF0C0000000000000000000000000000000000000000000000000000000000000000000000000000000000000000000000000000000000000000000000000000000000000000000000000000E3F820000480001008035100DA
:80178000084421220004800010080340000800012080040000000000000000000000000000000020000480001000824400080001200004800010000248000820012000041098F80000000000000000000000000000000000004000000000000000000008000000000000000000000000000000000000000000000100000000000000000017
:80180000000000000000020000000000000040FC00000000000000000000000000000000000000000000000000000000000000000000000000000000000000000000000000000000000000000001000000000000000000000000000000000088FE0000000000000000000000000000000000000000000000000000000000000000000000A3
:8018800000000000000000000000000000000040000010000000000000040000000000000000000000000000D8FE00000000000000000800002000000000000000000000000000000000000000000000000000000000000000000000000000000000000000000000000000000000000000000000000000000018FD00000000000000000081
:8019000000000000000000000000000000000000000000000000000000000000000000000000000000000000000000000004000008000000000000002000008000100002000068FA020000000000000000000000000000000000000000000000000000000000000000000000000000000000000000000000000000800000000000000002C3
:8019800000000000000000000000000000000018FD00000000000000000000000004000010000000000000000000000000000000000000000000000000000000000000000000000000000000000000000000000000000800800000000000000040FB200000000000000804002010000000200000000002100000000000400000000000002D
:801A0000000000000000000000000000400008000000000080000004020000000001000000010210000200000088FE2800000000000002100008400200000C00000000021000000000000001000000000000000000000000000000000000012000000000000002000108000000140400044000034A400900000040FF0000200004000010C8
:801A8000020140080100402000000000000080000000010100000000000000000000000000000000000001040700000000040000000801000000500A0012028300004800000000D0FD000000000000000080000000000080000000000000008000000000000000000000000000000000000000000000000000000000000004000000000015
:801B00000000000000000040800000000000000098FF0000108000000008040020100000001000000000000000000000820000000000000000000000000000000000008000000800000000000000000402000000000000020201000004000000805DF900000000000000000000000008040000000000000000000000000000000000000037
:801B8000000000000000000000000000000000000000000000000000040000000000000000000000000000000000D0FF000000000000000000000000000000000000000000000000000000000000000000000000000000000000000000000000000000000000000000000000000000000000000002000000000000B8FF0000000000000059
:801C0000000000000000000000000000000000000000000000000000000000000000000000000000000000000000000000000000000100000000000000000000000000000000000088FF10000000000000000000000000000000000000000000000000000000000000000000000000000000000000000000000000000000000000000000CC
:801C80000000000000000000000400000000000000CCFF000000000000000000000000000000400000006000000000000000000000000000000000000000000000000000000000000000000000000000000000000000000100000000000020000000B8FA000000000020000000000000000000000000000000000000000000000000000082
:801D00000000000000000000000000000000000000000000000000000100000000000000000000000000000000000088FD00200000000000000000000000000000000080000400000000000000002000000000000000000000000000000040000000002020040000120000400008000100000480001000024000000090F90000000000C01B
:801D800000000000000000000000000000000000000000000000000000000000000000000000000000000000000000000000000000000000000000000000000200000000010000000030FA00000000000000000000000000000000000000000000000000010000000000000000000000000000000000000000000000008000000000000035
:801E000000000000000000000000000000000000008098FE00000000000000000000000000000000000000000000010000000000000000000000000000000000000000000000000000000000000000000000000000000000000000000000000000000098FE00000000000000010000000000000000000000000000080000000000000000AC
:801E8000000000000000000000000000000000000000000000000000000000000000000000000000000000000000000010FE000008000000000000000000000000000000000000000000000000000000000000000000000000000000000000000000000000000000000000100800000000000000000000000000000000C4FB0000100000E5
:801F00001000000000000000000000000000000000000000000000000000000000000000000000000000000000000000000000000000000000000000000000000000000000000000000089FE0000000000000000000000000400000000000000000000000000000000000000000000000000000000000000000000000000000000000000C6
:801F800000000000000000000000000000000000000000D8FB00008000000000000000000000000000000000000000000000000004000000000000000000000000000000000000000000000000000000000000000000000000000000000000000000000050FB0000000000000000000000000000000000000000000000000000002100001E
:80200000000000000000000000000000000000000000048000000000000000000000000000000000000000000000000000E0FA000000000000000000000000100000000000000000000000000000000000000000000000000000000000000000000000000000000000000000020000000000000000400000000000000000E8FD00000000CB
:80208000000000000000000000080000000000000000000000000000000000000000000000000000000000000000000000000000002000000000000000000200000000000000000000000030FD00000000000000000000000000000010080000000000000000008000000000000000000000000000000000000000000000000000080000E9
:80210000000021040000000040000000000000000000000070FA00000008000000000000000000000000080000020080000000000000000000000000000000000000000000000000000008000000000000000000000000000000110000020000000000000080FF0000000000800100040000100000000000000000000000000000010000CE
:802180000000000000000000000000000000000000000000000000000000000000000000000000000000000000000000000050FF00000400000000000000000000000000000000000000000000000000000000000000000000000000000000000000000000000000040000000004000000000000000000000000000000000098FF080000E5
:8022000000000000000000000000000000000000000000000000000000000000000000000000000000000000000000000000000000100000000000000000000000000000000000000000040080FA0000100000000000000000000000000000000000000000000004000000000000000000000000000000000000000000000002400000007A
:802280000000000202000000000000000000000000000000009AFE00001000000000000001000000000000000000000000002000000200000000000000000000000000000000000000000000000000000000200000020000000040000800010000000000000048FC08400008022000080400201000020000000040000880000000014000A7
:802300000000000000000000000000000000000000800000000000000000000000048000100002000000048020000000000000C0FD000009A000100002900008400008000000001000024000100001240000000000000000000000000000000000002000000014400000000010000124000480002100D492000A80000000000020FE002048
:80238000102294C0001002086008448040000000802030290040010C0200200800000000000000000000000000000000416000004000080002200008000120042420400D16420029800901040698FA00001000002000000000100002402000000000200000000000040200000400000000000000000000000000000000400000004000089D
:802400000000200000000000000000000804000000000000000080F9000001008140000404002040000000000000400008000010000200001000000000000000000000000000000000800010000000000000010000048000101001000000108100100082000008D8FE100000000000000000000000020000000000000000000000000000DA
:80248000020000000000000000000000000000000000000000000000000000000000000000000000000000004100000000004000CCFA000000000000000100000000101000081000000003000200000040000000000000000000000000000000000000000000000020000000000000200000000000A0000000000000000000000030FA000B
:80250000000800004000000000000000000000000000010000000000122000000000000000000000000000000000000000000000000002000000000000010000000000000000000000000000000028F800000000000000000000000000000000000000000000000000000000000000000000000000000000000000000000000000000000BD
:80258000100000000000000000000100000000000000000100000088FE00000000000000000000000000000000040000000000000000000000000000000000000000000000000000000000000000000000000000000000020010000000000000000000000000000088F90000000000000000000000000000000400000000000000000000A8
:802600008000000000000000000000000000000000000000000000000000000000000000000000000000000000000100000000000040FB02000000000000000000000000000000200000000000000000000000000000000000000000000000000000000000000000000000004000000000000000000000000000000000000000000098FBA9
:80268000000000000000000000000000000000000000200000000000000000000000000000000000000000000000000000000000000000000000000000000000000000000200000000000000000000B8FD000000000000000000000000000000040000000000000000000000000000000000000000000000000000000000000000000000FF
:8027000080008000000000000000000000000000000000000000008058FB00000000000000000000000000000000000010000000000000010000000000000000000000000000000000000000000000000000000000000000000000000000000000000000000001000098FF00000000000000000000000000000000000000000000000000DD
:80278000000000000000000000000000000000000000000000000000000000000000000000000000000000000000000000000000000098FF0000000000000000000000000000000000000000000000000000000600000000000000000000000000000000000000000000000000000000000820000000000000000000000000000000009480
:80280000FF000000000090480200000800000000340000000002000000000120000000000000000000000000000000000000000000000000000040000000000000000000000002400000000100000000E0FE00000000004000000000000000000030000000000000000000000000000000000000000000000000000000000000000000004F
:8028800000000000000000000000000000000000000000000000000000A8FB0000000000800000040000000000003C000000000000000000000000000000000000000000000000000000000000000000000000000080000000000000000000000000000000000200000088FB0000000000C0425800000000000000300000000000000000E6
:80290000002C02000000000000000000000000000000000000000000000000000000230000000000000000000000000000008C0000000080FD000000000080000010006002000000300000000098000000004000080000000000000000000000000000000000000000000000000000080000000000000000000098001001008004000000C6
:8029800068FD0000000000F0401E0000781000000038000000001E100000000F684000000000000000000000000000000000000000000000000000C003020000000000000000001EC80000000F00000000A8FA0000000000C0001800006000000000300000000018000000000C800100000000000000000000000000000000000000000016
:802A00000000000000030000000000000000000018000300000C0000000070FD0000000000E0029904006000000000300000000018000000004C82450000000000000000000000000000000000000000000000000000930000000000000000000018004300004C02000000C8FC000000000090020200006800000000000000000000000089
:802A80000000012000044200000000000000000000000000000000000000001000000000000001A001000000000000400000000100000000D4FC000000000000400000006000000000000000000000000000000000000000000000000000000C00000000000000060000000000000000000000008001000000000000000000000000000079
:802B00000048FB0000000000C000000000002000000000000000000000000000000000000000000000000000080000000000000004000000000000000000000000884100000000000000000000000200000068F9000000000080221810006000000000000000000000000000002C820502100000000000000000000000000000000000000B
:802B80000000000000000000000C8011000000000000000000008C000000005BF90000000000C04800100060020000000000000000000000000000040000210000000000000000000000000000000000000000C0020000000000408051000000000000002000004010000000C9FB0000000000F0001E00001820000000000000000000006C
:802C00000000000FE0010D000000000000000000000000000000000000000000F04000000000000FE801000000000000C00001000F0000000090F80000000000C0201800006000000000000000000000000000000C800100000000000000000000000000000000000000000000C00000000000000C0000000000000000000301000C000016
:802C80000000B3FD0000000000C0041804001021000000000000000000000000000C824110410000000000000000000000000000000000000000C00000000000000C8201010000000000000300000C0200000098F9100000000010000200000800000000040000000042440000000120080400000000000000000000000000000000000020
:802D00000000000000004000000000A00100000000000040000000000000000010F9000000000000000000006000000000000000000000000000000000000100000000000000000000000000000000000000000000000000000000000000000000000000000000000000000000F8F800000000000000000400000000000000000000001EB6
:802D800010000000000081000800000000000000000000000000000000000000000000000080000000808100000000000000000200000000000008FF0C00000000C0825800000021000000000000000000000000000000093001000000000000000000000000000000000000000000000000230000008005000000000000001300000000F4
:802E000000000050F904000000000042000800602400000030400000000804430000409000021200000000000000000000000000000000000000000000000000010000009000000000000000000100000000000098FC0000000000F0001E000078000000003C0000000014C003000003E0003C0000000000000000000000000000000000B6
:802E800000000000000000C0030000006000000000000000C00300000000000000A0FE0C00000000C0001800006000000000300000000018040300000C00003000000000000000000000000000000000000000000000000000030000008001000000000000000300000000000000C0F90000000000C0005904006020000000300000000072
:802F000018000300008C0420B0080000000000000000000000000000000000000000000000008B0000000044000000000000008B0000000000000078FA00000000001000020000080000000000000000000200000000012010340000000000000000000000000000000000000400000000000000000000200000000000000040000000011C
:802F80000000000030FB0000000000C000000000600000000000000000000000000000000000010000000000000000000000000000000000000000000000000000000000000000000000000000000000000000000070FC00000000000040000400002000000000000000000000000000000001310000000000000000000000000000000083
:8030000000000000000000000000000000000000000000000000000000000200000098FE0C00000000C0085800006004000000000000000000000000002C0209300A000000000000000000000000000000000000000000000000000000000000000000000000000000008C0000000028FC0400000000C02280080060040000000000000035
:80308000008020000000808490801000000000000000000000000000000000003021000000000000000000801100000000000000000000000400000060F90000000000F0001E00007810000000000000000006000000000FE0000C0000000000000000000000000000000000003C00000000000000000000E001010000000000C000020056
:803100000F0000000058FF0C00000000C0001800006000000000000000000018100000000C00000000000000000000000000000000000000000030000000000000000000000040000000000000000300000C0000000030FD000000000020401805001042000000000000000018010000008C0240801000000000000000000000000000007F
:8031800000000030000000000000000000000010000000000000009300008C02000000E0F8000000000090080A010048000020000000000000020000000001203104000000000000000000000000000000000000000000000000400000000020000000000000004000000001000000004CFF000000000000400804000040000000000000BB
:8032000000000000000000008001000000000000000000000000000000000000000000000000000000000000000000000000000000000000000000000088FA0000000000C0000600006040000000000000000000000000000000000008000000000000000000000000000000000000000000000000000000000000010000000000000000DC
:80328000000000000000E0FE0C0000000080248002004000000000000000000018050000002C82083201000000000000000000000000000000000000000000000000000000008005000000000000002304000000000000A3FA0400000000C044800000602200800900000000000009000000400481001100000000000000000000000000BD
:803300000000000000000000000000200000000080000000000000000001008000000000B9FB1800000000F000041000780000E08100000000001E000000000F60003C000000000000000000000000000000000000000000000000C000010000E001000000000000C00300000304000000A0F80800000000C00010040060100080010000E9
:8033800000000018040000000C02013008000000000000000000000000000000000000000000000000030100008041000000000000008300000C0000000063FC0000000000C0849000006000008001000000000018010000008C00103102000000000000000000000000000000000000000000000000230000008011000000000000002343
:8034000000004C0400000000FD0000000000D000020000080000000000000000001A00000000012011340000000000000000000000000000000000000000000000000000000000A001000000000000400008000100000000F0FF0000000000C00000000000000000000000000000000000000000804100000000000000000000000000004B
:80348000000000000000000000000000000000008001000000000000000000000000000000D0FA00000000000040000000000000000000000000001804000000000080080000000000000000000000000000000000000000000000000000000000C00100000000000000000000000200000068FE0C00000000C000000000000000000000A8
:803500000000000058000000002C8200840800000000000000000000000000000000000000000000000000000000A001000000000000000000008C00000000CAFC0400000000C0008120006020000000000000000000020000000001013100000000000000000000000000000000000000000000000000000000008001000000000000002B
:80358000406020200000000070F9180000000030000600007800000000000000000006000000000F6000082000000000000000000000000000000000000000000000000000000000C001000000000000C00078000F0800000008FA0800000000C0001810006000000000000000000000100000000C0201340000000000000000000000006A
:8036000000000000000000000000000000000000008001000000000000000360000C02000000D9FF000000000020425800006000000000000000000000000000002C0000010500000000000000000000000000000000000000000000000000000000A001000000000000008360002C0000000020FA20000000001000020000080000200010
:8036800004000000000200000000002000040100000000000000000000000000000000000000000000000000000000200004000010000040030000010000000014FC0000000000C00000000060000000003000000000000000000000000000080000000000000000000000000000000000000000000000000000000020000000000000009F
:80370000000000000000000000E0FF000001000000000004000020000000011000000000000000000080013C00000000000000000000000000000000000000000000000000000000006000000000000000C0000000000200000068FD8C010000000042580000600000800130000000001805000000000050801000000000000000000000BB
:803780000000000000000000000000000000000000002000000000000000008800008C000000003BFB0488000000C048400000600C000020B0100000008008000000008045900800000000000000000000000000000000000000000000000000000000804530040000000000030000400400000021FCF801000000F0001E1000780000E08E
:80380000013C000000001E0000000000E001280000000000000000000000000000000000000000000000000000000000C0013C0000300000800001000F0000000050F98841000000C0001804006000008041300000000018040000000080413008000000000000000000000000000000000000000000000000000000008001300000000022
:8038800000000300000C0200000053FE8001000000C048180000102100800108400000001800000000008011300200000000000000000000000000000000000000000000000000000000800130000000000000A000000C0000000080F920000000001000024000080000000004000000001A0000000001200004000000000000000000005D
:8039000000000000000000000000001000004000000000A001000000D0000040030000000000000078FE000000000000000000000000000000000000000000000000000000000000000000000000000000000000000000000000000000000000000000008001000000C0000000000000000000000040FF000000000000000000000000004D
:803980000000000000000004040000000080010000000000000000000000000000000000000000000000000000800000008041000000C04000C08000000000000000D0FA0000000000C0821810006021000000304000000002010000002C02480000000000000000001000000000000000080000000000000000230000008011000000C093
:803A0000020000200000000000000028FD8081000000008280081360240000003012000000580000000020805100010200000000000000010000000000000000000000C0020000200100008051000000C0100000130000000000000000FDE001000000F0001EC0037A000000003C0000000004100000000FE8010C20040000000000001086
:803A8000020000000000000800000000F04000C003000000E001000000F0000080000100000000000008FD8001000000C040180403602000000030200000001A000000000C820131800400000000000050020000000000000800000000C000000083000000000000000000000000830000000000000068FD8001000000C0049800036002DD
:803B0000000000B00000000000020000004C800130080400000000000000020000000000000000000000C0000000130000008001010000C08000000800000000000000C0F80000000000000000000000000000000000000000000100000000000000020400000000000000020000000000000000000000000000000000000000000000002A
:803B80000000000000000000000000008CFE20000480001000024000080001200004800010000250000800012000042000000000000000000000000000000020000480001000024000080001008004800010000240000800012000040020FF0000000000000000000000000000000000000000000000000000000000000000000000000048
:803C0000000000000000000000000000000000000000000000000000000000000000000000000000000098FF2C0004800010000240000800012000048000100000400008000120000000000000000000000000000000000000200004800010000240000800010050048000100002400008000120000400E3FB040000000000004800000009
:803C80000000000080000000000802000000000000901000000000000000000000000000000000000000000000000000000000000400000000000000210000000000000059FF3800048000100002480008000120000490001000024000080001200004000000000000000000000000000000002000048000100002400008000120400480E8
:803D00000010000240000A00012000040030FA080000000000000000000000000000000000000000000000000000000000000000000000000000000000000000000000000000000000000000000000000000000000000000000000000000A3FC20000480001000024000080001200004A200100002400008000120000400000000000000AD
:803D8000000000000000000000200004800010000240000800012050048000100002000008000120000400F8FA00000000000000000400000000000000000000000008000000000004001000000000000000000000000000000000000000000000000000000000000000000000000000000100000000000080FA0000000000000000000004
:803E0000000000000000000000000000000000000000000000000000000000000000000000000000000000000000000000000000000000000000000000000000000000000098FF000000000000000000000000000000002000000000000000000000000000000000000000000000000000000000000000000000000000000000000000008B
:803E80000000000000000000000000000000B8FD020000000000000000000000000000000000000000000000000000000000000000000000000000000000000000000000000000000000000000000000000000000000000000000000000000B8FD000000000000000000000000000000000000000000000000000000000000000000000056
:803F00000000000000000000000000000000000000000000000000008000000000400000000000000000000050FB00000000000000000000000000000000000000000000000000000000000000000000000000000000000000000000000000000000000000000000000000000000000000000000100000000088FE04000000040000000098
:803F800000080000000000000000000008010000000400000000000000000000000000000000000000000000000000000000000000000000000100000004000000000000000048FA000001000000000000000000004000000800000000000000000100400004000000000000000000000000000000000000000000000000010008000000CE
:80400000000000000010000002100000000400E0FE00000100010000080000100080A1000020000000008C002000410503012000000000000000000000000000000000000000000000804200004000000000000100000208000240000000040000F90800100000400004444400001280040000000000180022424501010030000000000012
:8040800000000000000000000000000000100080001080000000000008802200000000000200900A001400000488FD000004000040000010000000004000000000000004000000000000000400000000000000000000000000000000000010000000000000000000000000000000000000000000000000000000D8FB060000000000000038
:8041000000000200000000000000000008800008000004000800000000000000000000000000000000000000008000200000000000000000080000000000020000400000000020F0FB00000000000000000000400000000000000000000000000000000040000000000000000000000000000000000000000000000000000000000000002C
:804180000000000000000000000000000000000098FB00000000000000020000000000000000000000000000000000000000000000000000000000000000000000000000000000000000000000000000000000000000000000040000000000000098F90000000000201000000008000000000000000000000000000000000010000000004D
:8042000000000000000000000000000000000000000000000000000000000000000000000000000000000000000010FC100000000000001000000000000000000000000002000000000000000000000000000000000000000000000000000000000000000000000000000000000000000000000000000000000000FCFA000000000000001A
:80428000010000000000000000000000000000000000000000010800000000000000000000000000000000000000000000000004000000000000000000000000000000100000000048FA000000000000000000000000000000000000000000000000000040000000000000000000000000000000000000000000000000000000000000001E
:804300000000000000000000400000000000000000D8FB400000000000000000001000000000000400000000000000000000000000000000000000000000000000000000000000000000000000000000000000000000000000000000000000000000C8FA1800000000000000000000000000000000000000000000000000000000000000FC
:804380000000000000000000000000000000000000000000000000000000000000000000000000000000000000000080FF00000000000000000000000000000100000000000000000000000000000000000000000000000000000000000000000000000000000000000000002000000000000000000000000000000088FD00000000000098
:8044000000000000000100000000000000000000000000000000000000000000000000000000000000000000000000000000000000000000000000000000000000000000000000008044FB0000000000400000000000000000000000000000000000000000000000000000000000000000000000000000000000000000000000000000003C
:8044800000000000000000000000000000000000000098FB000000000000000000000000000000000000000000000000000000000000000000000000000000000000000000000000000000000000010000000002000000000000000004000000000000E8FE000000000000000000000000000000000000000002000000000000000000003A
:804500000000000000000000000000000000000000000000000000000000000000000000000000000000000000000000B8FF00000000000001000000000000000000000000000000000000000000000000000000000000000000000000000000000000000000000000000000000000000000000000010000000000000088FF0000000000FB
:804580000000000000000000000000000000000000000000000000000000000000000000000000000000000000000000000000000000000000000000000000000000000000000000000098FF0000000000000000200000000000000000000000002000000000100000000000000000000000000000000000000000000000000000000000D4
:8046000000000000000000000000000000000000000000B8FC00000000000000000000000000000000000000000000000000002000000000000000000000000000000000000000000000000000000000000000000000000000000000020000000000000098FF0000000000000000000000000000000000000000404000000000000000004D
:80468000000000000000000000000000000000000000000000000000000000000000000000000000000000000000000000D8FB080000000000000008000000000000000000000000000000000002000000000000000000000000000000000000000000000000000000000000000200000000000000000800000000000000B8FD0000000016
:80470000002000000000100000000008000000000000000000000000001400000000000000000000000000000000000000000000000000000000000004000000000000000000000000000080F9000000000000010000000000000000100000000000000000000000004000000000000000000000000000000000000000000000000000001F
:80478000000000000000000040000000000000000000000098FA000000000000000000000020002000000000000000000000000100000000000000000000000000000000000000000000000000000000000000000000000000000000000000000000000000B8FE000000000000000000008000000000000000000000000000000000000070
:804800000000000000000000000000000000000000000000000000000000000000000000000000000000000000000000000090FF800000000000000804000000000000000000000008000000000002001000000000000000000000000000000000000000000000000000800000000000000000000000000000000402000000C0FA82000041
:80488000000000000000000000000080100000000000480000000040000000000000000000000000000000000000000000000020000000000000000040000000000002100000000000000000D8FF1A000100012000000000000000400000000000000080000000000001010000000000000000000000000000000000000000000000000455
:804900000040200000000000840000080000000000000000000AFE4003018000100050008000000020C0080000000000C8000000006200A1000000000000000000000000000000000000000000200080120008400000856080004400060800000A0400000000A8FE200000008000002A801440A00400211022008000180400D0A40440207E
:8049800020040000000000000000000000000000000000000404C000800002000000204420060D00004804420012001400000080FE00000000000000040000000002000020000000000208000000020000000000000000000000000000000000000000000000004000000000000000008000000000000210000010000000000018FF000055
:804A000000008000000000001000004020000000100010000010000000201020000000000000000000000000000000000000100480000000010000000000080802000000000102000000000000E8FF00000000000000000000000000000000000000000000000000080000000000000000000000000000000000000000000000000000002D
:804A80008000000000800000000000000080000000020000000010FD00000000008000000000400000000000200000000404000000060000082000000000000000000000000000000000000000000000008000000000400000000000000000000000020000000030FF080000000000004000000000000000000000000000000000000000D8
:804B0000000000000000000000000000000000000000000000000000000000000000000000000000000000000400000000000000F2FD000000000000200000000000000000000000000000020000000000800000000000000000000000000000000000000000040000000000000000000000000000000000800000000000000000D8F90249
:804B80000000000000000000800000000000000800000000040000000000000000000000000000000000000000000000000000000000000000000000000000000000000000000000000000000000F0F90000000000000000000000000000000000000000000000000000000000000000000000000000000000000000000000000000000040
:804C0000000000000000000000000010000000000100000000000098FF000000000000800400000000000000000000000000000000000200000000000000000000000000000000000000000000000000000000000000004000000000000000000000000000000080D0FD100000000000000000000000000000000000000000000000000069
:804C800000040000000000000000000000000000000000000000000000000000000000000000000000000000000000000010000000C8FA020000000080000000000000000000000000000000000000000000800020000000000000000000000000000000000000000000000000000000000000000000000010000010000000000000B0FFED
:804D000000000000004040000000200000000020000000000000000000000000040000000000000000000000000000000000000000008000000000000000000000000000000000000000000000000050FD0000000000000000020000000000000000000000000000000000400002000000000000000000000000000000000000000000005E
:804D8000000000000000000000000000000000400000000000000000DAFB00040000000080000000000000000400000000000000000000000000200000000000000000000000000000000000000000000000000000000020000000000000000000000000000000000058F9A0012440000000000000080000000000000000001A000000005E
:804E0000000000000000000000000000000000000000000000000000000000000000000000000000000000000201000000000000000020FC800110000000000000000000000000000000000018000000000000000000000000000000000000000000000000000000000000000000000000000000000000000000040000000000000000D88E
:804E8000FAE0012020000000000000000000000000000000001C000000000000000000000000000000000000000000000000000000000000000000000000000000000000000006000000000000000000F8FDA0013002000000000000602000000000000000001A000000000000000000000000000000000000000000000000000000000013
:804F00000000000000000000000000000000001804000000000000000018FF000020020000000000000040000000000000000000000000000000000000000000000000000000000000000000000000000000000000000000000000000000000014000000000000000000F8FA60403C10000000000000780000000000000000000604000028
:804F8000000000000000000000000000000000000000000000000000000000000000000000000000000000000010000000000000000000B0FA0000300800000000000060000000000000000000000000000000000000000000000000000000000000000000000000000000000000000000000000000000000000100000000000000000004F
:80500000F0FB200038020000000000006012000000000000000002000000000000000000000000000000000000000000000000000000000000000000000000000000000000000008000000000000000000F8F90000042100000000000000000D000000000000001A0000000000000000000000000000000000000000000000000000000032
:80508000000000000000000000000000000000004200000000000000000030FE0000100000000000000000000C0000000000000018000000000000000000000000000000000C00000000000000060000000000000000000000000000000000000000040000000000000000F8FD0000100800000000000000000F000000000000001E0000BC
:8051000000000000000000000000000000000800000000000000040000000000000000000000000000000000000006000000000000000000A0FC0000B00000000000000000000D000000000000001A00000000000000000000000000000000000000000000000000000000000000000000000000000000000000005A04000000000000004C
:80518000003BFA00003040000000000000000080000000000000000001000000000000000000000000000000000000000000000000000000000000000000000000000000000000001400000000000000000019FD00003C00000000000000000003020000000000000604000000000000000000000000000000000000000000000000000014
:8052000000000000000000000000000000000000001000000000000000000048F8000030080000000000000000000000000000000000000000000000000000000000000000000000000000000000000000000000000000000000000000000000000010000000000000000000A3FE00003000000000000000000001000000000000000000C4
:80528000000000000000000000000000000000000000000000000000000000000000000000000000000000000000000800000000000000000008FD0000000000000000000000000D00000000000000122000000000000000000000000000000000000000000000000000000000000000000000000000000000000000020000000000000060
:805300000000E0FB0000000000000000000000000C000000000000000800000000000000000000000000000000000000000000000000000000000000000000000000000000000000000000000000000000000050FB0000000000000000000000000C02000000000000101000000000000000000000000000000000000000000000000000C5
:805380000000000000000000000000000000000000001E00000000000000000020F90C000000000000000000000040000000000000001801000000000000000000000000000000000000000000000000000000000000000000000000000000000000001A000000000000000000A0FA0400000000000000000000000C00000000000000103D
:80540000010000000000000000000000000000000000000000000000000000000000000000000000000000000000000014000000000000000000C0FE1800000000000000000000000D000000000000001E08000000000000000000000000000000000000000000000000000000000000000000000000000000000000000800000000000006
:80548000000000B0FB08000000000000000000000000000000000000001808000000000000000000000000000000000000000000000000000000000000000000000000000000000000000800000000000000000098FE0000000000000000000000000C000000000000009C0000000000000000000000000000000000000000000000000093
:80550000000000000000000000000000000000000000001000000000000000000098FB00000000000000000000000001000000000000009210000000000000000000000000000000000000000000000000000000000000000000000000000000800000001200000000000000000018FE00000000000000000000000000000000000000003D
:805580000000000000000000000000000000000000000000000000000000000000000000000000000000000000000600000800000000000000000078FF0000000000000000000000000A0000000000000018000000000000000000000000000000000000000000000000000000000000000000000000000000008007000014000000000069
:805600000000000008FD0C000000000000000000000005000000000000001004000000000000000000000000000000000000000000000000000000000000000000000000000000000000000800000000000000000062F9040000000000000000000000860200000000000018200000000000000000000000000000000000000000000000D9
:8056800000000000000000000000000000000000000300000C00000000000000000068FE18000000000000000000000009000000000000001E00000000000000000000000000000000000000000000000000000000000000000000000000000000000400001400000000000000000078FE0800000000000000000000000802000000000056
:805700000018000000000000000000000000000000000000000000000000000000000000000000000000000000000004000008000000000000000000C9FD000000000000000000000000040000000000000098020000000000000000000000000000000000000000000000000000000000000000000000000000000002000010000000008F
:805780000000000000D0F9000034000000000000000000010000340000000012200000000D000000000000000000000000000000000000000000000000000000000000000000000080100100000000000000000000006CF9000030000000000000000000000000300000000008000000000C000000000000000000000000000000000000CE
:8058000000000000000000000000000000000000000000000000000000000000000000A0F80000380000000000000000000A0000380000000010100000000F0000000000000000000000000000000000000000000000000000000000000000000000800101000000000000000000000098F90C00340000000000000000000500003400005B
:80588000000018010000000D00000000000000000000000000000000000000000000000000000000000000000000000016000000000000000000000000FBFE0400000900000000000000008602000009000000101000000040020000000000000000000000000000000000000000000000000000000000000000000000050000000000006E
:8059000000000000000099FB18000C0000000000000000000900000C000000001E000000000300000000000000000000000000000000000000000000000000000000000000000000000004000000000000000000000000D6FE0800000000000000000000000802000000000000180000000000000000000000000000000000000000000037
:8059800000000000000000000000000000000000000000040000000000000000000000007AFE00000400000000000000000004000004000000009C080000000100000000000000000000000000000000000000000000000000000000000000000000000002000000000000000000000000B8FF000034000000000000000000090000040080
:805A00000000009210000000000000000000000000000000000000000000000000000000001000000000000000000000804001000000000000000000000020FC000030000000000000000000040000000000000000000000000000000000000000000000000000000000000000000000000000000000000000000000000000000000000063
:805A800000000000000000D8F80000300800000000000000000A000000100000001800000000000000000000000000000000000000000000000000000000000000000000000000000000800101000000000000000000000020FF0C000001000000000000000005000030010000005010000000000000000000000000000000000000000028
:805B0000000000000000000000000000000000000000008006000000000000000000000000D8FB040030060000000000000000860200001200000018200000000000000000000000000000000000000000000000000000000000100000000000000000000005000000000000000000000000A8F818000C0000000000000000000B00003CA0
:805B8000000000001E000000000000000000000000000000000000000000000000000000000030000000000000000000000004000000000000000000000000A0FA0800000000000000000000000402003008000000180800000000000000000000000000000000000000000000000000000000C0200000000000000000000004000000006F
:805C0000000000000000000008FC000080200000000000000000080000B000000000180100000000000000000000000000000000000000000000000000000000C0040000000000000000000002000000000000000000000000F0FFA00134800600001A400068000D0000048006D00012200000000D00003400000000000000000000000003
:805C8000000000000000340000D000000000000000000000800001000000000000000000000004FB8001300006000018000060000C0000000006C00008000000000C000030000000000000000000000000000000000000300000C0000000000000000000000000000000000000000000000000B8F8E00138800700001E000078000C0000F9
:805D0000009007F00010100000000F000038000000000000000000000000000000000000380000F0000000000000000000008001010000000000000000000000E8FFAC0134800600001A000B69000C0000308106D00018010000000D000034000000000000000000000000000000000000340000D000000000000000000000802600000018
:805D800000000000000000000083F80450000A400100000500021400020000214001281000000000800200000A0000000000000000000000000000000000000A00C000000000000000000000000500000000000000000000000011FB78000C8001000006C00318000300003C800130001E040000000300000C000000000000000000000064
:805E0000000000000000000C0000E0000000000000000000000004000000000000000000000000A6FB0800000000000000008300000000003008000000180000000000000000000000000000000000000000000000000000000000C0000000000000000000000004000000000000000000000000F2FB000000000000000000030000000002
:805E80000030000000009C1000000000000004000000000000000000000000000000000000040000C000000000000000000000000200000000000000000000000028FD000004800600001A40006800010000348006D000921000000000000034000000000000000000000000000000000000340000D00000000000000D0000008000000099
:805F000000000000000000000000E0F8000000000600001800006000000000300006C000000000000000000030000000000000000000000000000000000000300000C00000000000000C000000000002000000000000000000000020FC000000100700001C000070000002003C0007E00018100000000000003C000000000000000000005F
:805F800000000000000000003C0000E00000000000000F000000800100000000000000000000000088F80C0030810600001A000B6900200000348006D000100000000000000034000000000000000010000000000000000800340000D00000000000000C000000802602000000000000000000000000F90400800000010000040001104C87
:8060000000000008000120182000000000000000080200000000000000010000000000000000000800C00000000000000C000000000500000000000000000000000038FF18003C9001000006C00318000302000C800130001E000000000000000C0004000000000000100200000000000008000C0000E00000000000000E000000000400D6
:806080000000000000000000000000D0F80800300800000000008300000002000000000000180000000000000000800400000000000050020000000000000800000000D00000000000000C000000000400000000000000000000000098FC00003081000000020013080080000000800010005820000000000000000004000000000000004F
:80610000020000000000000000000000D00000000000000C000000000200000000000000000000000018FC000000000000000000000000000000000000000000000000000000000000040000000000000002000000000000000000000000280000000000000000000000000000000000000000000000D0FB000000000010000040000000E2
:80618000002000000000000000400008000020000000000000000000000000000000000000200000800010000240000800012000048000100002400008000120000400D8FD004000080000000000000000000000000000020000000000000000000010000000000000000000000000000000000000000000000000000000000000000000CA
:80620000000000000000000000000000F0F82C000480A01000425000080A21220084904010488250000800812800040100000000000000000000000000000020000491000040024000080001200004800010000240000800012000040013FC0400000000000000000000000000000000000000000000000000000000000000000000000045
:80628000000000000000000000000000004022000000000000040000000202000808000000000000000041FA1800000000100000400000000020000000000000004000080001200000000000000000000000000000000000002000008000100002400008000020000400001000004000080001200004009EFB0800000800010000040000AF
:80630000100004000008000120000000000000040000080000000000000000000000000000000000000800000000000000000000000000000000000000000000000000009AFB20888480201000824000080281200004822010048244000800812000040000000000000000000000000000000020000480001000024000080000240004801B
:8063800000100002400008000120000400C8F800004000000000000000000000000000000000000000000000000000000000000000000000000000000000000000000000000000000000000000000000000000000000000000000000000098FB0000000000000000000000000000000000000000000000000000000000000000000000008B
:8064000000000000000000000000000000000000000000000000000000000000000000000000000000000098FF00000000000000000000000000000000000000000000000000000000000000000000000000000000000000000000000000000000000000000000000000000000000000000000000000000098FF00020000000000000000EC
:80648000000000000000000000004000000000000000000000000000000000000000000000000000000000000000000000000000000000000000000000000000000000000098F900000000000000000000000000000000000000000000000000000000000000000000000000000000000000000000000000000000000000000000000000CB
:80650000000000000000000000000000000098FF04000000000000000000000000000000000000000000000000000000000000000000000000000000000000000000000000000000000000000000000000000800000000000000000000000058FB08000000000000000000000000000000000000000000000000010000000000000000001C
:806580000000000000000000000000000000000000000000000000000000000000000000000000000000000090FE004000000000000000000000040000000000008002000000000000000000000000000000000000000000000000000000000000000000000000000000000001000000000000000000000000A0FF000001050000000000A1
:8066000000001001000000000000800200000000020000000000000000000000000000000000000000000000000000000000C000000000008000400000000000000000000000E0FC020000000000000000000000000200000000000000042025000002000000000000000000000000000000000000000000000000000000000000000000DA
:80668000000000000200A8260500000000000034F900000000000000000000000000020000000000000004000800000400000000000000000000000000000000000000000000000000000000000000000000000000000000000000000000000018F90A0000000000000000000000000000000000000000000000000000000000000000006B
:806700000000000000000000000000000000000000000000000000000000000000000000000100000000000000B0FC00000800000000000000000000000008000000000000000000000000000000000000000000000000000000000000000000000000000000000000000000000000000000000000000000000010FF00000000000000004D
:8067800000020000000000000000000000000000000000000000000000000000000000000000000000000000000000000000000000000000000000000000000000000000000000B8FD0000000000000000000000000000000000000000000000000000000000000000000000000000000000000000000000000000000000000000000000E2
:806800000000000000000000000000000000000098FF100000000000000000000000000000000000000000000000000000000000000000000000000000000000000000000000000000000000000000000000000000000000000000000000000000CCFB12000000000000000000000000000000000000000000000000000000000000000098
:8068800000000000000000000000000000000000000000000000000000000000000000000000000000000000008064F900000000000000000000000000000000000000000000000000000000000000000000000000000000000000000000000000000000000000000000000000000000000000000000000000000098FF0000000000000024
:806900000000000000000000000000000000000000000000000000000000000000000000000000000000000000000000000000000000000000000001000004000000000000000000C8FF000000000000000000000000000000000000000000000000000000000000000000000000000000000000000000000000000000000000000000004B
:80698000000000000000000000000000000000008010FF00000000000000000000000000000000000000000000000000000000000000000000000000000000000000000000000000000000000000000000000000000000000000000000000000000098FF000000000000000000000000000000200000000000000000000000000000000051
:806A000000000000000000000000000000000000000000000000000000000000000000000000000000000000000000B8FF00000000000000000000000000000000000000000000000000000000000000000000000000000000000000000000000000000000000000000000000000000000000000000000000000000098FF000000000000C8
:806A800000000000000000000000000000000008000000000000000000000000000000000000000000000000000000000000000000000000000000000000000000000000000000000090FF000000000000000000000000000000000000000000000000000000000000000000000000000000000000000000000000000000000000000000FF
:806B000000000000000000000000000000000000000098FF00000000000000000000000000000000000000000000000000000000000000000000000000000000000000000000000000000000000000000000000000000000000000000000000000000098FF00000000000000000000000000000000000000000000000000000000000000E7
:806B8000000000000000000000000000000000000000000000000000000000000000000000000000000000000000000098FF00000000000000000000000000000000000000000000000000000000000000000000000000000000000000000000000000000000000000000000000000000000000000000000000000000098FF000004000063
:806C000000000000000000000000000000000000000000000000000000000000000000000000000000000000000000000000000000000000000000000000000000000000000000000000D8FF00000000000000000000000000000000000000000000000000000000000000000000000000000000000000000000000000000000000000003D
:806C80000000000000000000000000000000000000000098FF00000000000000000000000000000000000000002000000000000000000000000000000000000000000000000000000000000001000000000010000000000000000000000000000000000098FC00000000000000000000000000000000000000000000000000000000000038
:806D000000000000000000000000000000000000000000000000000000000000000000000000000000000000000000000098FF000000000000000000000000000000000000000000000000000002000000000000000000000000000000000000000000000000000000000000000000000000000000000000000000000000B8FF00000008BB
:806D8000000000000000080004000000000000000000000000040000000000000000000000000000000000000000000000001000000000000000000000000000000000000000000000000058FE00000000000000000000000000000000000000000020000000000000000000000000000000000000000000000000000000000000000000FD
:806E00000000000000000000000000000000000000000000B8FF08000000000000000000000000000000000000000000000000000000000000000000000000000000000000000000000000000000000000000000000000000000000000000000000000000090FF0E0000000020000000000000000000100000000000000040000000000145
:806E80000000000000000000000000000000000000000000020000000000000000000000000000000000000000000000008068FC1C000000020000080000200000000000000040000000000000000000000000000000000000000000000000000000000000000000000002000000000000000000000000000008000000000000F9003300F0
:806F0000860C2018020301080080010068000010008002001010280080000000000000000000000000000000000000000000150000004000000000000060001400000000000040000000000068FD80500106020100088000200000000010080000180000A00502000001300800000000000000000000000000000020020000104000000084
:806F800002000004000000800424010000000000000000000088FB40400000810000040000100000000010080000000000000200000000100400000000000000000000000000000000000000002000000000000004000000000000000000000000000000000028F80000000800000000000000000000000000000020000000000000400070
:80700000100000000000000000000000000000000000000000000000008000000000000000000400000000000000000000000068F810000000000000000000000000000000000000004400000000000000080000000000000000000000000000000000000000000000000000000000000000000000000000000000000000000004FF0000BD
:807080000000000000000400000000000000000000002004000000000000000000000000000000000000000000000000004000000000000000000000000000000000000000000000000000000098FD0000002000000000800800010000000000000000001000000000000000000000000000000000000000000000000000000000000000DA
:807100000000000000000000000000000000000000000000000038FF00000000000000000000000000000008040000000000000000000000000000000000000000000000000000000000000000000000000000000000000000000000000000000000000000000090FB1E000000000000000000000000000000000000000000000000000023
:80718000000000000000000000000000000000000000000000000000000000000000000000000000000000000000000000000000C2FB00000000000000000000000000000000000200000800000000000000000000000000000000000000000000000000000000000000000000000000000000000000000000000000000000000038FF0091
:80720000000000000000000000000000000000000080000000000000000000000000000000000000000000000000000000000000000000000000000000000000000000000000000000000000008090FF020000000000000000000000000000000000000000000000000000000000000000000000000000000000000000000000000000007D
:807280000000000000000000000000000000000000000000000000B8FD000000000000000000000000000000000000000000000000000000000000000000000000000000000000000000000000000000000000000000020000000000000000000000000000000000B8FD00002084000000000000000000000000000000000202000000007A
:807300000000000000000000000000000000000000000000000000000000000000000000000000000000000000000000000000000058FB140000000000000000008000000000000000000000000000000000000000000000000000000000000000000000000000000000000000000000000000000000000000000000000000000000C0FB6B
:8073800000000000000000000000000000000000000000000000000000000000000000000000000000000000000000000000000000000000000000000000000000000000000000000000000000000098FF000000000010005250000000000000000000902802400068000020040400000000000000000000000000000000A0010000001009
:8074000000004008090001200034800000000240000000000000000058F8000000000000000800030000000000000000C00000100060000000000100000000000000000000000000000000800100000000000000000000000000300000000018000000000000000000C0FB00000000000000101000020000000000000000001004006000FE
:8074800000008100000000000000000000000000000000008001000000C000000002000003600030000001000000800000000000000008FC0000000000000018000B00000000000000004042100183600000000100000000000000000000000000000000008001000000002800000A01000120003000260000182013000000000000006040
:80750000FF0000000000C00810090B01000000000000008008080100011400804030020000000000000000000000000000000004000000C02200001100112C801102014002009804000100000000000010F90000000000F0201EC003000000000000000030200ED003180000E0003C200000000000000000000000000000006040000000C1
:80758000F00000C00119000FE4010C880700001EC00300000000000000B0FE0000000000C00018000301000000000000008020000803000000000030000000000000000000000000000000000000000000C02000000060000C800100000600001800030000000000000058FE0000000000C0005CA020000000000000000000040001930034
:807600000000001032000000000000000000000000000000000000000000C00800001062240C800100002601008408930000000000000000F900000000001000125100000000201101000010001A400000000120042502000000000000000200000000000000210000804011820040080A22002000000000000012000000000020002406DD
:80768000A8FC0000000000C000000000000000800000000000001800000000000000101000000000000000000000000000000000000000000000000000000000000000000000000008000000000000100090FB000000000000801800000100000001000000300018000000000300012820000000000000000000000000000000000000009D
:807700000481200000024010000000010000000018040000000000002010B0F80000000000C00050042300000080910000001000180000000001002134020000000000000000000000000000008085000024800400008A4004008001000000000010000000000000003002C3FA0000000000C00458100B0200000005000000C08480042034
:8077800000004C84082101000000000000000000000000000000009000004240040000212200000004000000000018210000000080112000B9FF0000000000F0201EC003000000E001010000F00006C00001000FE0003C10000000000000000000000000000000E001008003724000C001382000E00101000000001E0000000000E0813CFF
:8078000010EEF80000000000C0001804030000008081000000C00000008300000C000030000000000000000000000000000000008001000000010000000000200080010000000000180000000000800130009AFF00000000002044980043000000C005000000C00000002300000C0084BC200000000000000000000000000000008041001A
:8078800000400014000040000000804100000000001809000000008001382268FA0000000000900002400008000020090080000000924800000000200926210000000000000000000000000000002000008024D100004000482400200000800000000240000000000000241100FA00000000000040000000000000008000000000001800DE
:8079000000000000800100000000000000000000000000000000000000000006C0000000006000000000000000000000000000000000000000A0FB0000000000C00000000000000080010000000000000000000000004030000000000000000000000000000000006000000000C00000C000000000804100000001000000800000000000F2
:807980003008A8FE0C00000000800459080000000000290000060400081083000000800820400000000000000000000000000000002000000002C200004000202200000000002600005808130000000000A00090FD0400000000C088000893000C00801101000002009004080000000091300200000000000000000000000000000080056B
:807A00000000040120000043401200804100001000000020100000000000300618F91800000000F0001EC003180000E001008007000006C00302000060003C10000000000000000400000000000000E501018001300000C003180000E00100800704001EC00302000000003C0070FF0800000000C0201800036000008001010006000010B8
:807A800000030000000001300000000000000000100000000000000080010000040100000003402000808100000600001800030000000000300888FE0000000000C0021802036021008005000016010080108B00000000043105000000000000000000000000000000800100000000000000030004008009000016010098028B00000000DB
:807B000000300058FB0000048000D000024000000000A0010080001020024008020000A00124080000000000000012000000000000002940008006108400400268000D200004800000000240004841000000000040FA0000300000C00018000000000080010000000000000000000000800110000000000000000008000000000000000863
:807B800000000006000000000362000C000000000000000000002000000000000080FE00003C0000000000000000000000000000068100180000000000800120080000000000000000000000000000000101000006800000000060000C00000D0000010000008040200000000000C0FB0800000000C010182000000000000000001080208F
:807C0000001110010000800130000000000000000010000000000000000845000006808200002161000C800104002600005808136004000000000023FF0000180046C008580463000000001001000641025820100100000040A0000000000000000002000000000000008108000000418800000A00120000883006000200800020410C00D5
:807C80000000000089F8000020800732401EC003000000600000800770401EC00000000060003C10000000000000001400000000000000E080008001700000C000190003E2013C800700001ED003780000000000001EFD0400200006C0401800030000000000000006002018080002000000003020000000000000000000000000000000A0
:807D00000200000000000000000201000080013000060000180003600000000000008AFC0000100006200884080300000000900000A600001800010000000000380100000000000000000000000000000000400000000010000008000000805130004601001821A37081000000000068FE00002400001000124000000000201125A200D0D0
:807D80000002400000000D2005240A00000000000000220000000000000031113480009010004062080000A00100000000001A000048220020310400F0FE0000100000C0000008030000008000100000C00000000001000C808100000000000000000020000000000000008A41300000C00000000300000080010000000000180000000067
:807E0000008000000098FC00002C000000401800000000000001200000C00006000001000C00003100000000000000000200000000000000000030000002000000001A0000800100000000000000006010000081000098FF000010000000089004030400008091301206C40002002000000C8010202008000000000000880100000000008F
:807E8000008290300016404800000108000080010000000000180200400100801100006BFE0000180000C0181821A300000000892011100008580020020080003130880000000000000000000000000000000405800840822000000A604000000000000000005810006041000011300001FA0000280000F0001EC003000000E0013C800743
:807F000034201EC80000000362003C0004000000000000020200000000000061400C8007300000C08078000060400000000000060000780000E0813C108EFB0000100000C0801800030000008001300006010018000202000000013110000000000000001000000000000000044100000681800000026200000000000000000018080060ED
:807F8000100080013100BAFE0000200000C00898A010010000C009BA204600001800080000000004B000040000000000000C020000000000000008000046000200000860000000000000000000040100600200C0093000D8F8300000000010001A40020000002009248120010002400000000020000480000000000000004000000000006E
:808000000000252104800090180040000800002000000000000002400008000020890400A0FB0000000000C0001800000100000080001000000000000000000000000000020000000000000A000000000000008201000000C200000000000000000000000000001800000000000000000030FC0000000000000000100300000080013000D2
:8080800004000000000000000000000C8000000000000000000400000000000008000C00040180000003000000000000000000000008800000008041000030FF0C00000000C0105800220100000001211104080000000000000000000080000000000000004A00000000000000849004002440000000800000000000000000000000011368
:808100006021000001B010BBFD8481000000C082980023040000801131222204000000600000000010300202000000000000000100000000000000053042428002000093000400005000000000001803080042008031002059FFF801000000F00006D003000000E0013C8003000006C40000000060403C0800000000000000100000000080
:8081800000000061403C8003328000C003181000600000000000001EC0037A0000E0013C00B6FB8801000000C040181003000000800130100000001800830000008001308004000000000000020100000000000008013000008080000003604000800100000000001808836020008041300092F98001000000200804009300000080813044
:80820000001001009802230000008049300001000000000000000100000000000000203000A000080000A36004008085000000000058000B6002008009301000FD100000000090440240030000000000048000100002400008000020000400040000000000000600000000000000303000800010001A400008000020080080000000024035
:80828000100900012000040010FE00000000000000180003000000000000000000000000000000000000000001000000000000A40000000000000010000000000000180000000000004000000000001800000000000000000000FE0000000000C000001000020000000000000000001800001800008001001002000000000000000100005E
:8083000000000000010100000002001C0000601000000101000001000000000000000000000060F80C00000000804200000B0000000000000000C08080048308000000403001000000000000000400000000000000004500001600001A0000000100000900002600001802400000008085B01073FE0400000000C0185810030100000000F8
:808380000004100148580010602100804900120100000000000090000000000000008208000020000400052060100080000000200000981020620C8C04100102C1FE1800000000F0001EC00000000000000C8001F0001EC4037A0000E0013C00000000000000000000000000000000E080008007342006C080780000E040008007040006C7
:80840000C00078000FE0013C201EFD0800000000C0001810030100000000300006C220180083600000800130080000000000000004000000000000000400000006C1000000036000000000000006010018080060000C80013010F2FB0000000000C0889880200000000000302206C00018080360000080453000000000000000000000001A
:8084800000000000000028000006C020020093604000004000000600001C011261000C80913000F0FC100000800010000240000000010000048014100002400000000020000400000000000000000000000000000000200000800010001A40030800002011008000000092480008000020000400B8FB0000000000000000000300000000B7
:808500000000000601000000000000000000000000000000000000000000000000000000000000000000180003000000804100000000000000000000000000000068FB000000000000000000000100000000000000040018040000000060000010000000000000000000000000000000000000800130001E000360000000000000000000F2
:8085800018000000000000000000D0F90C0000000000005808200000000000000042C08040008300000020003001000000000000001000000000000000888500800010001A0003001000804800000000005004006021008085000070FF0400000016C20240000B02000C0000002144080418052001000080210040020000000000001001B3
:808600000000000000000808000016C04200040860010000010100C000001803200002000004320068FD1800008007F0401ED00300000F04000C8001F0801EC003000000E0013C00050000000000009002000000000000E801018007F20006C080781000600000800100001EC000792000E0013C10B8FB0800000006C00018080302000CFE
:808680000000300804C120180083000000800130080600000000000014030000000000008A41000006C0000000006000000001000006000018008360000080013100C0FD0000000006C00018010300000C0000300040C004180513000000800130010400000000000008020000000000008409000006C000000000608000005000000602ED
:8087000000180503600A0080053000F8F810000000000000000000000000000000000000000000000000000000000000000000000000000000000000000000000000000000000000000000000000000000000000000000000000000088FF200004800010000240000800012000048000100002400008000120000000000000000000000213
:808780000000000000000021000480001000004000080001200004800010000240000800012000040088FA00000000000000000000000000000000000000000000000000000000001000000000000000000000000000000000000000000000000000000000000000000000000000000000000000000098FE2C000480001000024000080026
:8088000001200004800010000240000800012000040200000000000000000000000000000020000480001000424800080001200004800010000240000800012000040003FC040000000000000000000000000000000000400008000020000480000000000000000000000000000000000000800010000240000000012000048000100000F2
:8088800000000000000000000000000069FC380000900010000240000800012000048000100002400008000120000400000000000000000000000000000000200004800010000040000800012000048000100002400008000120000400B6FB08000000000000000000000000000000000000000000000000000000001000000000000000E4
:808900000000000000000000000000000000000004000000000000000000000000000000000000000000F2FC20008490001000024000080001200004800010000240000800012000040200000000000000000000000000000020000480001000024000080001200004800010000240000800012000040020FF000000000000000000000010
:808980000000000001000000000000000000000000000000000000000020000000000000000000000000000000000000002000000000000000000000000080000000000028FC000000000000000000000000000000000000000000000000000000000000000000020000000000000000000000000000000000000000000000000000000090
:808A000000000000000000000000000000B8FD00000000000000000000000000000000000000000000002000000020800000000000000080000000000000004000000000009010000002000100000000000000000000000000000000000098FA0000000000000000000000000000000000000010000000000000400000200010000000000C
:808A800000000008000000000000000000080020000000000008000000000000000000000000000000000074FD00000000000000001000000000000000000000000008000000000000000000000002000040000000000000A00000000000000000000040000000000000000000000000000000000000000098FE08000000000000000000F5
:808B00000000100000000001000000000000000000000000000000000000000000000000000000000000200000000000000000000000000000000000000000000000000000A1FE00000020000000000000000000000000000000000204014000000000000000000000000000000000000000000080000000800000000001080000020100B2
:808B80000000010000008140200004000000A0F9000000000000000200000000000000100000010000000008000001001000000000000000000000000000000000004010000240000010000000000040000801200000000002000000000000C0FB00000010A080010A00002000000000140000040004880018008009280400000000000036
:808C000000000000000000000000C0000580A01200009000101000442801A00012000080001320000400000860F90000148020800050400000100401218108A480208042C120001C0A09A40000000000000000000000000000000000009000A4000000004040000C0200345A02003838048760000481000021B0F8080010000000000000C6
:808C800000004002000000200000200000020900080200000000000000000000000000000000000000000400000000000000000008010020200200400888000900080001008039FD000000000010000800000000004800010002420000044000000400010400000000000000000000000000000000000000000201000000002200040000DB
:808D00001000000020040001200000080000005CFB000000000000000000000000000000000000000020200000000000000800000000000000000000000000000800000100000000000000000000000000000000000000000000000000000000B8FC0000000000000000040000000020000000000000000000000000000000000000000016
:808D80001000000000000000000000000000000000000000000000000000000000000000000000000000000000E8FC00000000000000000000000000000000000000000000000000000000000000004000000000000010000800000000000000000000000000000000000000000000000000000000000000000008FB1000400000000000D4
:808E00000008000000000000000000000000000000000001000800000004000000000000000000000000000000001000000000010000000100000000000020000000000000000024FA0000000000008000000000000000000000000000000004000000000000000000000000000000000000000400002000000000000000000000000000E5
:808E80000000000000000000040000000004000038FF00000000000000000000000000000000000000000A00000000000000000000000000020000000000000000000000000000000000000000000000000000000000000000000000000000000038FD0000000000000000000008000000800000000000004000000000000000000000002A
:808F0000000000000000000000000000000000000000000000004000000000008000000000000000000000004000D0FF08000000000000000000000000000000000000000400000000000000000000000000000000000000000010400000000000000000000000000800000000000000000000000000000000000066FD000000000000005B
:808F8000000000000000000000000000000000000000000000000000000000000000000080000000000000000000004000000000000000000004000000000002000000000000000078FD00000000000010000000000000000480000000000000000000042000000000004000000000010000000000000100000000000002004008000000F2
:809000000000010000000000020000000000000080C8F900000000000000000000000000000000000000000000000000000000000000000000000000000000000000000000000000000000000000000000000000000000000000004000000000000098FB000000000000000000000000000040108000000000000000000000000000000009
:8090800000010000008000000010000000000000000400000000001000000004000000000000000000000000000000C8FE00000000020000008000000000000000000000000000000000000000000000000000000000000000000000000000000000000000000000000000000000000000000000000000000000000010FD00000000000072
:80910000000000000000008000080000000010000000000000000000000000000000000000000000000000000000000000000000000000000000000000000002000000000000000000B8FE00000000000000000000000000000000000002400000000000000000000000000008000000000000000000000000000000000000004001000014
:80918000000000000000000000000000000000000000E0FC00000000000000000000000000000000000000000000000000000000000000000000080000000000000004000000400000000000000000000000000000000000000000000000000000000010FF0000000000000000000000000000000000000000000000000000000000000038
:80920000000000000000000000000000000000000000000000000000000000000000000000000000001000000001000088FF00000000004000400001000000000000000020000080010000000000080000000000000020000000000000000040000000010000000000000000000000000100000880012800008000100088FC000000000005
:809280000000020000000000000000000000200000800000000000000000000000000000000000000000000000400000000100000000000000000000000001000800800000000000001078FB000000000000012C00040000000000000000800000000400000000000000000000400000000000000001000000000000000000000000000089
:8093000000000040000000000020000400000200000000B0F8400000000000000000010000000000000000000000000000000000004000008000000000000000400000000000000000000000000000000000000000000008000000000000000000000008C0FA00002000000000000000000000000000008000000000000000000020100004
:8093800000000000000000000000000000000000000000000010100000000000000000000000000000000000000000000020FD00000000000000000000000000000000000000000000000000000000002000000000000000000000000000000000000000080000000000000000000000000000000004000000000000000072FB0000000097
:80940000000000000000000000000000000001000000800000000000000000000000000000000000000000000000000000000000000000800000800000000001000000800000000000088098FF004008800000000000000000000000000802001000100120200100002100000000080000200000000004000010000000000000000000003A
:809480000000000000048000100004080008080000002000E4F8000100000020801090000240000800040400002000400010000042000000000000000000200000000004002000004000080404000000000000000040000004000002100000400000400080FCFF20C00800011080025000024000082804300100C080CA00382002A8800890
:809500000000000010000030000000000C042008800001A0008416080001200A00000009800120000618005061000000690510FB00480100031000100001D00008002108040280001406C305080820C102500000000212C000000000000002101080E0022405501448000B0500000200010084402808048040118057020000E0FA000001BD
:8095800080000000008000000000000000000100000004010200000000010000000000004000000000000002001020000100004000024000000000080000000020201008800040000400000068FD000000000000000400001000024020000400200004820001400280000000000000000440000000000000000000000001080200100000A2
:80960000010000000000008000040000000008000008000000A0FD100000000010010002400000008000000000000000004000000000000000000000000000000000000000000000000000000000000000000000004000000000000002500000080020000400CCFD00000000000000100000000000000040080000000000000000000000B6
:80968000240400000000000000000000000000000000000000000000000000000000000000000000001000004000000001200010FE000000000000000020000000000001200000000000040000000000000010000000000000000000000000000000000000000000000000000000000004000000000000000000000000000200A8FA0000C6
:809700000000000000000000000000000004040000000000000000000040020080000000000000004000000000000000000000000000000002000000000000000000000000000000000000000038FB160000000000200000000000000002000000000000000000000000000000000000000000000000000000000000000000000000000072
:809780000000000000000000000000001000000000000020008040F800000000000000000000000000000000000000000000000000000000000000000000000000000000000008000000010080000000000000200000000000000000000000000000000000000030FC000000000000100040000000000000000001000000800000000000DB
:8098000000000000000000000000000000000000000000000000000000000000000000000000000100000080000000000000800080FB00000000000002001000020000000000000000000008080000000000000000000008000000000000000002100000000000000000000000000000000000000000000010080000000000000098FD0081
:809880000000000000004400000000000000000800000000000000000020003000002000400000000000000020000000000000000200000000000000000000000000000000000008000000000000C4F80000000000000000000040000000000000000400000000000000000000000400020000000000020201000000000000000000000037
:809900000000000000000000000000000000000000080000004000B0FC00000000080000000402000000002000000000000000000000000000000000000004000000000000000000000000000000000000000000000000000000000000000000000000000002000010F9000000000080000000000000000000000000000000000000000036
:809980000000000000000000000000000000000001000020000000000000000000004000000000000000000000000000000004000060FE000000801402000200004821000000008000D000000000000000A00104000000000000000000000000000000000000008010128402400000000120000080C010000240010A00212000840088F843
:809A000000000000020000000000200000000000000000000000000000008001000000000000000000000000000000000000000000000000000000000000000000000000000210010840000400001090FE000000000400000008004000000000000000C00000000000000080013008000000000000000000000000000000000000000481FC
:809A8000400080000000000000000004000016C00058000B00002C00A0F8000000004602001800006022000000000000C002010000000000800180000000000000000000000000000000000000000044800000400000004C8409020000C4440800A02000040000100060FC0000000004020040080040040000000000860040000000000088
:809B00000000483008000000000000000000000000000000000000004240228004030100400090000016010414009050000A8011280058FF000000800700001E00007820000000008007300000000000000060003C000000000000000000000000000000000000008003720006800300000FE801008007F080108000400008E00121002841
:809B8000FA000000000600001808006000000000000006C020000000000000000030200000000000000000000000000000000000000000000018000300000C8001000006C10014100250200A0040280008FC00000000870000980000704400000000000600040000000000000000B0000000000000000000000000000000000000000000A7
:809C0000084418200300004C8249000046C02408000A2400040000100008FC00000080240000024082480000000000000000000000000000002008060000000000000000020000000000000001000080001000424800080001200000800010000240000800212000840060FB00000000000200180001002000000000000000000000000075
:809C800000000000000000000000000000000000000000000000000000000000000000000000000000000000000210000840000400001080FC000000000600000008826000000000000000000000000000000000410020000000000000000000000000000000000000000000001084000000000000000000000016000059000B00002C00EF
:809D000080FE0000000024080018010140240000000000000000000000000000001130000000000000000000000000000000000000000016080090400060404C84090200A6C0440800232000040044100023FC0000000016020098000B622100000000000000000000000000008008011000000000000000000000000000000000000000CE
:809D80004002000809030024200008000000020415000850000A0008280099FA000000800700001EC40178000000000000000000000000000000E0003C00000000000000000000000000000000000000800730200E808378000FE801018007F00010C0034200086040200006FE00000000060200180003600000000000000000000000004F
:809E0000000000000030000000000000000000000000000000000000000006C00000080360000C8001000006C00014000350000A00002800AAF80000000046000004881361080000000000000000000000000000008830080000000000000000000000000000000000000006C18880000360100C8241000006C1208808832082048029107B
:809E800000A8FE20000480000000124100482100000000000010000200006800012030844000000000000000000000000000000000000080449000024000080001200000800010000240010900212004860058FD0000000000000000080020000000000000000000000000600000000000000000000000000000000000000000000000008A
:809F00000006C140000000000000000000000000000210010840000400001050F90000001000000018040340000000000000000000060000600003000120000000000000000000000000000000000000000000002018C4000000000000000000000016C08058000B40002C0008FF0C0030000000001000036022000000000000C00201006D
:809F800000600001000521120000000000000000000000000000000000000002420200010060404C8409020016C84408000820000420841000C0F8842100010600009808834040000000000000004818040000028C8408100100000000000000000000000000000000000000248148580483002280048000001000021400A050000A000450
:80A00000290018FDE0013C900702001EC0037800000000000000F0001C000018100FE0001D08000000000000000A00000000000000010000800130001E800378000FE001008007F4801080004000084000200040FC8C0130000600001800836040000000000000C00018000000000C00000000000000000000000000000000000000040031
:80A08000000004818018000360000C8001000006C00014000250200A00002800F0FC800130220600001809037000000000000000C02218000000000C008000080000000000000000000000000000000800000020000898020360112C8245000016C12208088220010420911000C8FB000004800010001A40034800000000008000000002CE
:80A100000000080000200004000000000000000006000000000000000000048006D0001248002804012000008000100002400908002120008400C8FF0000300000C00018000300200000000000000000000000000000000000000000000000000010000000000000000000000006C000180000201000000000000000000210010940000494
:80A1800000001038F9000000200000800090036040000000000000000006000018000080010C0000000000000000020000000000000005000C0006C0000088001840000000000000000016800358000B40002800D8F90800300100C00498400340040000000000000000000000080000004404000000000000000004000000000000000141
:80A2000000040006C00008400000044C84090200A6C0440840002000042000140043FE0000301006C002180000612100000000008600001805006024008041B000000000000000001000000000000000100030202001221004230044401004000040020815800250000A8031280091F900000C8007F2800688007800000000008007000076
:80A280001C0000780000E0013C1000000000000000020000000000000008003C8001300006808310000FE001018007F000100002400008C0012000B6F80400300006C000180000600000000000000600001A0000600000804130000000000000000010000000000000000000300000000010080340000C8001000006C00014800250000A7B
:80A3000080012800DAFD0000B81006204244480060810000000000060000180000600000800130000000000000000008000000000000000500300000000040000340118C8251000046C128080901202004A001100090F91000A48000900202400048210000000000000000004003000000200034000000000000000000000000000000009A
:80A3800020000080001000024000080001A00000800010000240080800212000A400A8FB000000100600401800002000000000000000000000000300000000003000000000000000001200000000000000090000000000000000000000008040000000000002100009400004001010F0FC0000300000C40000C0004000000000000000005D
:80A4000000000003000000600030000000000000000000000000000000000000008001C0000080000000004000000000000016800258000B00802800A8F80C00A00826800041080060220000000000000000000003000000200030000400000000000002020000000000008289008000004000400060404C2480000016C84408400120005F
:80A4800004801114008BFE0400302006C08018101340840000000000000000000088000000801101010000000000000020000000000000001088000016C0440001130082800000000020020814800250000A00042800F1F800003C8007F1001E80837800000000000000000000C000000000E0010C08040000000000000402000000000053
:80A5000000E001008007F20006848378000F4880008007F080100002400008E001290006F90C00300806C00018000360400000000000000000000000000000800100000000000000000010000000000000008841000006C00018100360100C0201000006C12014800250000A804128004AF90000300111C214181003700100000000000085
:80A580000000000000000000800100800000000000000040000000000000008611000006C04218010360048C0041000046C00808110120080480112000A8FF000004800010000240004800000000000000100000400000000D2000040004000000000000100200000000000020000080001100024000080001A0040080001000024008084B
:80A60000002120001408B8FA000000000000000000000020000000000000000000000000000C00000000020000000000000401000000000000060000000000000000000000008040000000000002100009400004001000F8FC000000000000000008006000000000000000000000C00000000C00000080000000000000005000000000006B
:80A680000000600000000431001880000000004000000000000016800258000B00800C0028FB00000000160200180000400A000000000000C00201400000000C000000800000000000000050000000000000002A00000044100000440060404C2490000016C8440840012000048011000AEBFC0000301006C410002020602100000000009C
:80A70000000004000043000020000480000200000000000000010000000000008011010042C0429800930020801010000040084814800250000A0008020991F800003C8007F0001EC0007900000000000000F08000C00300000362400C08000000000000000400000000000000E201008003F2001E840378000F4000018007F000100002C6
:80A78000400008E0010800C6FF0000300006C0001810036220000000000000C020000003000000800130200200000000000050020000000000008201000000C00018000360100C0201000006C12014800250000A804120207AFD0000300026C2005800236004000000000000C002000003000000804130010400000000000080000000005A
:80A800000000008101000000C10018080360012C0051000016C0028820012024048005200290FD10000400000000125000482100000000000000001A000000000020012482000000000000001002000000000000080034804418001A400008000120300080020000024008080021A0019420C0F800000000000000180000200000000000C0
:80A88000000000001800000000008081300800000000000000040000000000000010003000060000180000000000000000800201000210000940008401100090FE00000000000000100080400000000000000000001C0000000000000001800200000000000050010000000000000000300000C000188000000000600000800700001680DF
:80A900000258000BE0010C2018F90C00000000000008020B602200000000000000001A00000000008010100A0000000000000000000000000000000400300002022418400060404C04280000000000084001200004A001000093FF04003010000000180210418000000000000000001800000000000049200101000000000000920000003D
:80A98000000000000100000124C10200048B0002400444000005000014800250000A8001002099F900003C000000000EC003780000000000000000001C000000000060000C1000000000000000000000000000000000000C8801F02006800378400F40000000040000100002400008C0010800FEFF0C003000000000180083600000000080
:80AA000000000000001A0000000000000120000000000000000004000000000000000400000004C28000000360100C0240000005000014900250200A80012000CAFD000030000000005C080370210000000000000000180000000000001082400000000000000000000000000000000000000010C00400000360000C00110000420100480E
:80AA8000000120020480012041E0FE100004000000005240004800000000244000D0001A000000000020110400000000000000000000000000000000A00100800010000240002812012000008000100002400848002120080500C0F80000000000000000080000200000003000000000180000000000808100000000000000000000000097
:80AB00000000000000800100000000000000002000000000008000010002100029400004000000A8FD000000100000001800806000000000000000C0001C0000000000000030000000000000000000000000000000008001000000C0000680001800000000008005000016C00258000B80000100A0FC0C00300000000090040B4042000062
:80AB800000101000C0021B0000000000801081080000000000000010000000000000008801000016082002400000214C8409020002C0440800012000040008302020FE040000060000001810206121000000A0100000401800000000000005300A0200000000000010010000000000000844000000C2281803A3000C00048800000500447E
:80AC000014800250000A80810012B8FF00003C000000001EC00378000000000C000030001C000000000060003D000500000000000090020000000000006800008007F0001E800310000FE001000004F000100002500008E0013C00A0F80C0030200000001804836000000000200000C02018000000000000013000060000000000001403A5
:80AC80000000000000000A00000006C12018000340100C8241000005C02014880250000A8001300828FF00003000000000580013604100000000400000041A0000000000002030050400000000000008020000000000000400000026C00818000340004C8009000002C10488000140210480493001F8FF00000000000000000001000000A6
:80AD00000000000000000080080000000000000000000000000000000000000000000000000000000000000000000000000000000010000040200000410080000000F0FA2000048000100002400008000120000480001000004000080001200004000000000000000002000000000000002100048000100002400008000120000480001159
:80AD80000002400008000120000400B8FD00000000000000000000000000000000000000000008000000000000000000000000000000000000000000000000000000000000000000000000000000000000000000000000000000000090FF200004800010000240000800012000048000100042400008000120000400000000000000000036
:80AE000000000000000000200004800010000240000800012000048000100002400008000120000400ABF800000000000000000009020000000000000000000809012000048000100000000000000000000000000000000080001000024000080011212100808400000200008808092122240484901069FE200004800010000200000800BC
:80AE8000012000048000100002400008000120000400000000000000000000000000000000200004800010000240000800012000048000140002400008000100000400D8FD00000000000000000000000000000000000000000000000000000000000000000000000000000000000000000000000000000000000000000000000000000053
:80AF0000000000000000000000000000ABFC200004800010000200000800012000048000100000400008000120000400000000000000000000000000000000200004800010000240000800012000048000100002400008000120400400F8FB00000000020400000000200000000000000000000000000000000000000000000000200000AF
:80AF80000000000000000000000000000000000080000000000000000000020020000000000000808000F8FD00000000000000000000000000000000000000000000000000000000000000000000000000000000000010000000000000000000000000000000000000000000000000000000000000000088FF000020000000000002000001
:80B0000000000000000000000000000000000000000000000000000000000000000000002000000000000000000000000000000000000000000010000004000020200000F8FC0000000000000000000000000000000000000000000000000000004020000010000400000000000800000000000000000000000000000000080000000000E4
:80B080000000002000000000000000000020FA00000000000000000800400800000000000000000000000000000000000000000002004000000000000008800000000000000000000000000000000000000000000000000800000000000078FD00000000080000000000000000000000200000000000000000000000000000000000000057
:80B1000000000000000000400000000000000000000000000000000000000000000000000000000000000070F9000000000020000000000020000100000000000008000000000400000000000000000000000000000000000000000000000002000000000000000280000002410004008100200204000000E8FA0000000000000000000085
:80B180004000000000200002000000080100000000410000000000000000000000000000000000000100000200000802000000040000000000202000000022100402000008F8F8800000000E2000000000283000040004800001200450000000062000010500000000000000000000000000000020000080A00200521400000001048000C6
:80B20000000132805480000B60030C001020E8FA000024800010001028430500000000000016410008000828088843002400000000000000000000000000000000000004004484004000206500080320100842C1201216C748A0040200005008F9000000000000000000020000000000000002840010000020000004000000000000000020
:80B2800000000000000000000000000000000000000000004000000200080404814000900002000402000080D8F90A0008000000001040800000000000000004000000000000080102001000000000000000000000000000000000000000000240000000002000040100010000400004080141000000000000E5F80000000000000000007E
:80B3000000000000000000000000000000000000000000000000000000000000000000000000080000000000000000200000000000000000000000000000000000004000000030F90000000000000000000008000000000000000000000000000000000000000000000000000000000000000000000000000000040000000000000000022E
:80B3800000000000000000000000000000000070FF00000000000000000000000000000000000000000000000000000042000000000000000000000000200000000000008000000000000000000000000000000000000000000040000000000010FF1000000000000000000400000000000000000000004000000000000000000000100049
:80B40000000000000000000000000000000000008000040000000010000000000000000008000020000000800074FA00000000000000000004000000000000000000000000000000000000000000000000000000000000000000000000000000000000040000080000000000000000000000000000000000000050FF0000000000000000C3
:80B4800000000020000000000000000000000000000000020200000000000000000000000000001000000000000000000000000000000000000000000040000000000000000000A8F80000000001000000000000000000000000000000000000000000000000400000000002000000000000000100000000000000000000000000000000F4
:80B500000000000000000000008000000000000000F9000000000000000200000000000000008000000000000000000200000000000000000000000000000000000000000200000000000000000000000000000000000100000000000000010000E6FB000000000000000000000000000000000000000000000000000000000000000001E8
:80B58000000000000000000000000000000000000040000000000000000000000000000000200000080000000000A0FB000000000000000000000000000000000000000000000010000000240000000000000000000000002000000000000400000440000000000000000000000000000000000010000000000000D8FD00000C00000000BB
:80B600000010400000000000000000000000000000000000000000000002000000000000000100000000000000000000000000002000008000000000000000000100000480001000CCFD0000000000000000000020000000000000000000040000000000000000000000000000000000000000000000000000000000000000000000000055
:80B680000000000000000000000000000000000000F8FD08000080000000000000008000000000000000000000000000000000000000000000000000000000000000000000000000000000080000000000000000000000000000000000000000008089FE02000000000000000000000000000000000000000000000000000000000000003C
:80B700000000000000000000000002000000000000000001000000000000000000000000000000000000000000000088FE00000000000000000000000000000000000000000000000000000000000000000000080000000000000000000000000000000000020000000000000000000000000000002000000000000010FF00000000000007
:80B7800000000000000000000000000000000000000000000000000000000000000000000000000000000000000000000000000000000000000000000000000000004000000000000098FB000000000000001080000000000000000000000000000000000000000000000000000000000000000000000000000000000000000000000000E6
:80B8000000200000000000000000000000000000000020FC04000000000000000000000000000000000020000800000000000000000000000002000000000000000000000100000000000000000001008002400000000020000000000000000000000090FE00000000000000000000000000000010000000200000000000000000000000BC
:80B88000000000000000000000000000100000000000000000000000001000024001000000200000000000000000001088F920000000001000000000000000000000000000000000000000000000000000000000000000000000000000000000000000000010000000000000080000000006800800022000080040200020FA0000000000BA
:80B9000000002400000000000000000000000000000000000000000000000000000000000000000020000000000000000000020000000000000003000000000000040010000000000024A8FE00000000000000000000000000000000000000000000000000000000000000000000040000000000000000000000000000000000000000009C
:80B980000000000000000000000000000000000000000098FB00000000000000080000000000000040000000000000000000002000000000000000000000000000000000000000000000000000000000000000000000000000000000000000000005000000F80000000000000020000000000000000000000000000000000000000000002F
:80BA000000000000000002000000000001000080000000000000000000000004024000000201200000800000000000020072FF202010200000000000800000002000000000000000480000000040000000000000080400200000000000042000004100000000001000002020000000100000102004080000000402001008E5FE040000001D
:80BA800001200000000022000040000000000000000400000000080000080000000804400000000000000020000000100000004008020000000402002080000080000001200001000008803EF9408008900010000000000B100060000006000018009800000000484000200000001806401000000000000160004080040014018006100063
:80BB000010200108000C801420C00C4C0028100304006C1008F90000005080804111000240000800211008001010900043650C048080025000000008048020000000000C03401800E122040421B0020240A009208340A00686C0200A2A0928B0040251505700FE000000000000000000000000000000100400000000800010000200010096
:80BB800000000000021000200000000004020010002000000001200000002000002280008000402010000110080402401000E0FF000000008040000400021000024020000000002002404040100000000000000000000040000000000004020810804008100400200008400010000800080802240000080000000080000008C0F81000004A
:80BC00000000000000000000100000000000002000010000000000000000000000000000000000000000000000000000000009000000000000000204000000010840000000000000000000000CF9000000000000A000800100090000000000000000000000000000000000000000000000000000000000000000000000000001000000000B
:80BC8000003000008000008001400000000000000000000800D8FC000080001400024000000000000000002000000008000000000000000004000000000000000000000000000000000000000000010000000000000080000000000004000840000000000200D0F9000028000480001400008000000000000000000000000000000000001D
:80BD00000000000000000000000000000000000000000000000000000002004001002000000000000000000000000000000000D8FA000000000000000200008000000000000000000000000000000000000000000000000400000000000000100000000000000008000000000000000000008000000000820000000000000000A8FB00004B
:80BD800080000000000000000000000000000000000000000000000000000000000100000000000080000000002000000000000000000000000000000000000000000000000000000020000000B8FE000000000000000000000040000000000000000000000000000000008800000000000000000000000000000000000000000200000082
:80BE00000000102000400000000000000000000000000000000048FE00000000000000000000000000000000000000000000000000000000000000000000000040000000000000000000000000000000020000000000100000000000000100010000008020000070FD000000080000000000000000000000000000000000000000000000A3
:80BE8000002000002000000000000000100000000000000000000000200000000000000000000000000000100000000000000000B0FF0000000000000008004000000000000000000000000000000000000004000C000200000000000600010000000000000000002000001000000000000000000000000000000000000000000418FD0861
:80BF0000000000000000000000080100000000000000000000000000000000000000000000000000000000000800000000000000000000000000000000000000000000000000000000000000008044FB00000000020000000000405000000000000000000000000000000000800000000000020000000000000000002000000000000000BD
:80BF80000000000000000000000000000000000000000000000000D0FCA0010000001000000000080000201001000000000200000000000000000000000000000000000000000000000000000000000000000000080000000000000000000200000000000000000008FD0000000000C00000000000000000000000000000000000000000BA
:80C000000000000000000000000000000000000000000000000000000000000000000000000000000000000000000000000000000010FB80410000000000000000000000000000000000000000000000000000000000000000000000000000000000000000000000000000000000004000000000000000000000000000000000000058FE5E
:80C080008005000000C010000000602000002000000000001804000000000000000000000000000000000000000000000000000000000000000000600000000000000000000000000000000000000040FB0088000000C008000000002000008800000000000009000000000000000000000000000000000000000000000000000000000093
:80C10000000000000022000000000000000040040000000000000000E8FA6000000000F040000000780000600000000000001E000000000000000000000000000000000000000000000000000000000000000000007800000000000000000006000000000000000000D0FF8001000000C040000000600000000000000000001800000000AB
:80C180000000000000000000000000000000000000000000000000000000000000006000000000000000000018080000000000000000D8FA004800000020080000006012008088000000000098040000000000000000000000000000000000000000000000000000000000000000006012000000000000000058000000000000000000900D
:80C20000F900000080001000000000080000000000802001000200000000000000000000000000000000000000000000000000000000000000000000080000000000000000001A000000000000000000C4F8000000000000000000000000000000000002000000000000000000000000000000000000000C00000000000000060000000098
:80C280000000000000000000000000000000000000000000000000000050FD00000000000040000000000000000000000400000000000000000000000000000000000000080000000000000004000000000000000000004000000000000000000000000000000000000050FF0000000000C0080000006020000000000020020000000000A8
:80C30000000000000000000000000000000000000000000000000000000000000000006000000000000000000080020000000000000000A3F80000000006C81800000000240000000000060100000100000000000000000000000000000000000000000000000000000000000000000000820000000000000000400000000000000000006C
:80C3800011FA0000008007F0000000007800000000008005000006080000000000000000000000000000000000000000000000000000000000000000007800000000000000000006080000000000000000C8FF0000000006C0000000006000000000000002010018040000000000000000000000000000000000000000000000000000001E
:80C400000000000000006000000000000000000000000000000000000000D3FA0000000006C0480000006010000000000016000058000000000000000000000000000000000000000000000000000000000000000000006010000000000000000000100000000000000000A8F91000000000100000400008000020000000000000020000F8
:80C480000000000000000000000000000000000000000000000020000000000000000000080000000000000000000200000000000000000088F8000000000000000000000000000080000000000000000000000000000000000000000000000000000000000000000000000000000000000000000000000000000000000000000000000012
:80C500000010FF00000000000000000080000000000000000000000000000000000000000000000000000000000000000000000000000000000000000000004000000000000000000000000000000000000018FB0C0000000000000000136020000020000000000018040000000000000000000000000000000000000000000000000000FE
:80C5800000000000000000600000000000000000000000000000000000000012FF0400000000C022000000022200008800000000000008000000000000000000000000000000000000000000000080090000000000000000000400000000000000000003000000000000000008FF0000000000F00000C003780000600000000000001E00F0
:80C600000000000000000000000000000000000000000000000000E08100000000000000007840000000000000000006000000000000000000A0FD0C00000000C000000003600000000001000000001800000000000000000000000000000000000000000000000080010000000000000000600000000000000000001804000000000000B9
:80C680000000A9F90000000000C00000008B6011008000000000000058040000000000000000000000000000000000000000000000800100000000000000006011000000000000000098000000000000000000E8F90000000000D000004000080000201000800000000240000000002000000000000000000000000000000000000000006B
:80C70000000000000000400008000000000000000000000000080000000000009CFF0000000000C000000000000000000001000000000000000000000000000000000000000000000000000000000000000000000000000000000000000000000000000000000000000000000000FA00000000000000000080000000000000000000000093
:80C7800000030000000000000000000000000000000000000000000000000000000000000080004000000000000000000000000010000000000088F80800000000C01000001360200000840000000000180408020000802100000000000000000000000000000000000000000000000000000B600000000000000000000000006000000065
:80C800000000003BF80000000000C00801000001820000200000C0000000104000000000900000000000000000000000000000000000000000000000000000000120000000000000000000000000220000000000E9F90000000000300000C003780000600000800100001EC000000000E00100000000000000000000000000000000000049
:80C8800000000000000000C0037800000000000000000000000078000000000000D8FB0400000000C04000000360000000410000060000180000000000800100000000000000000000000000000000000000000000000000000360000000000000000000000000600000000000004BFE000000000020080000A360140000100000A600006A
:80C9000018054000000080510000000000000000000000000000000000000000000000000000A3601400000000000000000000006014000000000070FD10000000001000004000080100A00100800000000240000000000000000000000000000000000000000000000000000000000000004000280000200000000010000200000000002B
:80C9800000000000F8FC0000000000C000000000001000800100000000000000000000000000000000000000000000000000000000000000000000000000000000001000000000000000000000000000000000000008FB000000000000400000800040000000000000000018000300000000000000000000000000000000000000000000C4
:80CA000000000000000000000080604000000000000000000000000000000000000038FB0C00000000000800001300020000000000460100180008020000000000000000000000000000000000000000000000000000000000000B6002000000000000000000000000000000000000F8F90400000000C018000020011100008000004002A3
:80CA80000018004000000000000000000000000000000000000000000000000000000000000000106402000030000000001800010000000000000000C8FD0000000000F00000C003180000600000800700001ED000000000000000000000000000000000000000000000000000000000000000C003784000600000000030000604000000A5
:80CB0000000000000028FF0C00000000C0000000834000000000010006010018040000000000000000000000000000000000000000000000000000000000000000836010008041000000C02018040000000000000000E0FA0000000000C0820000236008000004000046000018002001000000000000000000000000000000000000000001
:80CB800000000000000000000000236001008001000000C00418000000000000000000E8FB30000000001000004000080400208800800000000251030000000000000000000000000000000000000000000000000000000000024000080000000000000000000200000000000000000088FC0000000000C0000000002010000000000000A7
:80CC000000000000030000000000000000000000000000000000000000000000000000000000000000000000000000000000000000000000000000000030FB0000000000008000008040000000000000000000008003000000000000000000000000000000000000000000000000000000000000000060000000000000000000180000004B
:80CC8000000000000000B8FF0C00000000C000000013201200002000004601008048030000000000000000000000000000000000000000000000000000000000000000001000000000000000008002000000000000000042FA0430000000C004000040608100001001000002008008030000000000000000000000000000000000000000B5
:80CD00000000000000000000009800206010000000000000000000010000000000000000E8F86000000000F02000C0031800006000008007000006800300000000000000000000000000000000000000000000000000000000001EC800790000000000000000000610000000000000000090FE8C01000000C000000083604000000100007B
:80CD80000601001000030000000000000000000000000000000000000000000000000000000000180083600000000000000000000000000000000000000031F98081000000204400000B600000008800001600000002030000000000000000000000000000000000000000000000000000000000180013604200000000000000004008006C
:80CE000000000000000000F0F9300000000090000240086800002000008006000002008B0000002000000000000000000000000000000000000000000080000000004000680000201001000000000200000800000000000094F9000000000000401800814010000000000006000000000300000000000000000000000000000000000000E2
:80CE800000000000000000000000000000680000000000000000000808000000000000000090FF0000000000C0000010006000000000000000000000C00300000000000000000000000000000000000000000000000000000000000000807800000000010000000000100000000000000000C8F90C0000000080144000A06010000000007E
:80CF000000000000184403000000802100000000000000000000000000000000000000000086000000000B600000000400000000000000000000000000000093FB0408000000C088000288600200000800001001004010A0000000008800000000000000000000000000000000000000000000020000002061000000880000000000401002
:80CF800000000C0000000000B9F96000010000F00006C000781000604000800100001E8000000000E00100000000000000000000000000000000000000008007000000C003700000600000000000000600001800000000000058F88C81000000C000000080600000800100000600001804000000008041000000000000000000000000009B
:80D00000000000000000000006010000008360000000010000000000000800602000000000009BFA8009000000C024000220601100804500002602001800000000008001000000000000000000000000000000000000000000060000000003600000008800000000000001006002000000000060FB20000000001044004000080200200491
:80D08000018006000002400000000000000000000000000000000000000000000000000000000000000040600801000000000000108842100008000000000400B0F900000000000000000000001000800000000600000000000000000000000000000000000000000000000000000000000000000000000000001000000000000000000079
:80D10000000000000000000000F0FF00000000000000000000000000008000000700000000030000000000000000000000000000000000000000000000000000000000000000600000000000000000400000000010000000000050FE000000000000100000000040000008008006000018040300000000000000000000000000001000002B
:80D180000000000000080000000000000000100114000000000000000880080060000000000000E0FA00080000008088000020001400000400000600008020930000000000000002000000000000000100000000000000000000000000000012218100000000000000000011000024000000304008FD6000010000300000C000190000608C
:80D200008000000700001EC003000000000000000400000000000010020000000000000800000000000000C0005800000000000000304006000078000000003C0040FC800100000000000000034110000000000006000018040300000000000080040000000000005002000000000000080000000000000000002220000000000000808090
:80D2800010080060100000003000F8F88081000000004400000B600400002800000600009800A300000000000000040000000000000002000000000000000000000000000000006000000000000000000200010060020000003000C8FB10000000000000000000000000000000000000000000000000000000000004000000000000000295
:80D300000000000000000000000000000000000000120000000000000000000000000000000000008CFE20000480001000024000080001200004800010000240000800012000040000000000000000000000000000000020000480001000024000080001200004800010000240000800012000040098FF0000000000000000000000000036
:80D38000000000000000000000000000000000000000000000000000000000000000000000000000000000000000000000000000000000000000000000000000000098FF2C000480001000024000080001200004800010000240000800012000040000000000000000000000000000000020000480001000024000080001200004800010B5
:80D400000002400008000120000400E3F8040000000000000000000000000000000040000000000000000000000000000000000000000000000000000000000000000000000000000021000000000000000000000000000000000000D9FC20000480001000024000080001200004000014000200000A0001200004000000000000000000C0
:80D480000000000000000020000480001000024000000001200004800010000240000800012000040038FB0C0000000000000000000000000000000000010000008000000000000000000000000000000000000000000000000000000000000000000000000000000000000000000000000000000000FBF920000480001000024000080060
:80D5000001200004000010000240100800012000040000000000000000000000000000000020000480001000024000080001200004800010000240000800012000040080FE0000000000000000000000A000000000000002000000000000000000000000000000000000000000000000000000000000000000000000008000000000000035
:80D58000000000000000000000000000B8FF00000000000000000000000000000000000000000000000000000000000000000000000000000000000000000000000000000000000000002000000000000000000000000000000000000098FD00000000000000000000000000000000000000000000000000000000000000000000000000BF
:80D60000000000000000000000000000000000000000000000000000000000000000000000000000000098FF000000000000200000000000000000000000000000000000000000000000000000000000000000000000000000000000000000000000000000000000000000000000000000000000000000B8FF00000000000000000000003C
:80D680000000000000000000000000000000000000000000000000000000000000000000000000000000000000000000000000000000000000000000000000000000000098FF000000000000000000000000000000000000000000000000000000000000000000000000000000000000000000000000000000000000000000000000000093
:80D700000000000000000000000000000098FF00400000000000000000004000000000000000000000000000010000000000000000000000000000000000000080000000000000000000000000000000000000000000000000000000000058FE0000000000000000000000000000400000000400080400000000000000000000000000006B
:80D7800000000000000000000000000000000000000000000000000000000000000000800000000000000010FB02A80000008002000000002000800001000004005214000000020000000000000000000000000000000000000040000000000000000000000000000000000000000900500200040000000038F8080000000201000000404B
:80D8000000000040010000800A000400400000004000000000000000000000000000000000000000000000000000240000000000000000000000400040144010200000000470FA00000000010100000000000000000000000000000000000000000000000000000000000000000000000000000000000000000000000000000000000000C1
:80D880000000000000000000400000000000C8FE0800000000000000000002000080000000000100000040000000000000000000000000000000000000000000000000000000000000000000000000000000000000000000080000000000101DFC000000000000000000000000000000000000000000000000000000000000000000000026
:80D900000000000000000000000000000000000000000000000000000000000000000000000000000000000098FF00000000001000000000000000000000000000000000000000000000000000000000000000000000000000000000000000000000000000000000000000000000000000000000000000000098FE00000000000001000069
:80D9800000000000000000000000000000000000000000000000000000000000000000000000000000000000000000000000000000000000000000000000000000000000000088FE10000000000000000000000000000000000000000000000100000000000000000000000000000000000000000000000000000000000000000000000090
:80DA0000000000000000000000000000000000DCFB00400000000400000004000100000000000000002000000000000000000000000000000000000000000000000000000000000000000004000100000000000000000000000000000000002098FB00000000000000000000000000000000000000000000000000000000000000000000AE
:80DA8000000000000000000000000000000000000000000000000000000000000000000000000000000000000098FF20000000000000000000000000000000800000000000000000000000000000000000000000000000000000000000000000000000000000000000200000000010000200000800000000000020FD000000000000000098
:80DB00000000000000000000000000000000000000000000000000000000000000000000000000000000000000000000000000000000000000000000000000000000000000000098FF0000000000000000000000000000000000000000000000000000000000000000000000000000000000000000000001000000000010000000000000FD
:80DB80000000000000000000000000000000000088FF00000000000000000000000000000000000000000000000000000000000000000000000000000000000000000000000000000000000000000000000000000000000000000000000000000098FF00000000000000000000000000000000000000000000000000000000000000000007
:80DC0000000000000000000000000000000000000000000000002000000000000000000000000000000000000000A9FC00000000000000000000000000000000000000000000000000000000000000000000000000000000000000000000000000000000000000000000000000000000000000000000000000000098FF4000000000000008
:80DC800000000000000000000000000000000000000000000000000000000000000000000000000000000000000000000000000000000000000000000000000000100000000000009CFA000000000000000000000000000000000000000000000000000000000000000000000000000000000000000000000000000000000000000000007E
:80DD0000000000000000000000000000000000000098FF00000000000000000000000000000000000000000000000000000000000000000000000000000000000000000000000000000000000000000000000000000000000000000000000000000098FF000000000000000000000000000000000000000000000000000000000000000075
:80DD80000000000000000000000000000000000000000000000000000000000000000000000000000000000000000098FF000000000000000002000000000020000000000000400000000000000000000000000000000000000000000000000000000000000000000000000000000000000000000000000000000000F8FD000000000040F5
:80DE000000008000000000800100800000000800000000000000000000000000000000000000000000000000000000000000000001000000800000000040001800000000000000000058FB1000000000000002000100000040800000000000000000000000000000000000000000000000000000000000000000000000000000000000100A
:80DE8000000000000000000008080000000000000000FAFB00000000000081000000000000000200000000002040000000000000000000000000000000000000000000000000000000000000000004000000000200000000012000000000000000000008FB0000000000000000000080000000000000000000000000000000000000000090
:80DF0000000000000000000000000000000000000000000000000000000000000000000000000000000000000000000090FF000000000000000200000000002000000000000000000000000000000000000000000000000000000000000000000000000000000000000000000000000000000000000000000000000000B8FF080000000031
:80DF80000000000000000000000000000000000000000000000000000000000000000000000000000000000000000000000000000000000000000000000000000000000000000000008018FF000000000000000000002000000000000000000000208000000080000000000000000000000000000000000000000000000000000000002426
:80E000000000000000000000000000000000000000000038FB00000000000000000001000000000000000000000000000000000000000000000000000000000000000000000000000000000000000000000000000000000000000000000000000000000088FE920000000120000000000000000000000000000000000010000040002000C3
:80E080000000000000000000000000000000000000000000000000000000000000000000000000000400000000000000106AFE200010800010000080000000008003000000000000000A080000200004000000000000000000000000000000000000000000000000040A0000000000000000001400100000000000000020E8FE004080842F
:80E100008C0000080061600008806120000400000268060000080000105200000000000000000000000000000000010000000048916A020000800800485209800010026052000000001004E8FB008000000000000400011000004040000000000000000000000000000800000000000000000000000000000000000000000000000000009A
:80E18000000000000000000000000000000000000000100048FA00000020820000000080200002802008000100000080000000020000000000000000000000000000000000000040000000000000020201000000000000000080000810800800000000002048FC10000000001000000000100000200000000100000600020000000000003C
:80E20000000000000000000000000000000000000000000001000000C000102000002000000000100002000000000000000024FC9200000000000000000010000000000000010000040000000000400000000000000000000000000000000000000000000000000000800000010000000000000000000000300000000000803CFF00020006
:80E28000000000000080080800000000000000000040020000000000000000000000000000000000000000000000000000000000000000000000000000000000000000000000000000000000B0FB000000000000000000000000000000000000000000000000000000000000000000000000000000000000000000000000000000000000A1
:80E3000000000000000000000000000000000000000000000098FF00000000008000000000000000000000000000000000000000000000000000000000000000000000000000000000000000000000000000000000000000000000000000000000000000000010FF000000000000000000000001000000000000000000080000000000006E
:80E38000000000000000000000000000000000000000000000000000000000100000000000000000000000000000000000000090FE00000000000000000000000000000000000000000000000000002000000000000000000000000000000000000000000080000000000000000000000000000000000000000000000000000018FD0000CA
:80E400000000000002000000008000000400000000004000000000000000000000000000000000000000000000000000000000000000000008008000000400000000024200000000000000000090FF000000000000000000000000000000000000000000000000000000000000000000000000000000000000000000000000000000000077
:80E480000000000000000000000000000000000000000000000098FF020000000000000040000000000000000000000000000000000000000000000000000000000000000000000000000000000000000000000000000000000000000000000000000000000000B8F900000000000000000000000000000000000000000000000000000092
:80E5000000000000000000000000000000000000000000000000000000000000000000000000000000000000000000000000000098FF00000000000000000000000000000000000800000000000000000000000000000000000000000000000000000000000000000000000000000000000000000000000000000000000000000018FF06DF
:80E58000000000320200400000200120000000000000000000000000000000000000000000000000000000000000000000000080001002400000000000220400001000220000000002208204808061FD00000000B4900252000040012C20AD0000008002500000000000000000000000000000000000000000000000000000000000000092
:80E600000200000000080000000004810000000010080800012020F0F800000000000000000000000000000000000000012000000000000000000000000000000000000000000000000000000000000000000000000000000000000000000000000000000000000098FC00000000300002400000000120000C00000000000000000000006E
:80E680000000000000000000000000000000000000000000000000000000000000000000000000000000000000000000000000000038FA0015E002B4800A50012A4005A8002DA00254800A50012A4005A80015A0020000000000000000000000000000000015A0025C800BF0022AC005B80017E0025C800BF0032EC00FB80017E00270FD5A
:4FE70000A0089081336506CA0011280365A04C1581225006CAC011380245C0081401000000000000000000000000000000A0081401324006485411200364800C9001324006C80419201364800C900178FBFFFF0F
:00000001FF
